:020000040800F2
:10800000008001207DF80008C1950008C395000894
:10801000C5950008C7950008C99500080000000034
:10802000000000000000000000000000CB950008E8
:10803000CD95000800000000CF950008858B000852
:10804000C1F80008C1F80008C1F80008C1F800082C
:10805000C1F80008C1F80008C1F80008C1F800081C
:10806000C1F80008C1F80008C1F80008C1F800080C
:10807000C1F80008C1F80008C1F80008C1F80008FC
:10808000C1F80008C1F80008C1F80008C1F80008EC
:10809000C1F80008C1F80008C1F80008C1F80008DC
:1080A000C1F80008C1F80008C1F80008C1F80008CC
:1080B000C1F80008C1F80008C1F80008C1F80008BC
:1080C000C1F80008C1F80008C1F80008C1F80008AC
:1080D000C1F80008C1F80008C1F80008C1F800089C
:1080E000C1F80008C1F80008C1F80008C1F800088C
:1080F000C1F80008C1F80008C1F80008C1F800087C
:10810000C1F80008C1F80008C1F80008C1F800086B
:10811000C1F80008C1F80008C1F80008C1F800085B
:10812000C1F80008C1F80008C1F80008C1F800084B
:10813000C1F80008C1F80008C1F80008C1F800083B
:10814000C1F80008C1F80008C1F800083B92000817
:10815000C1F80008C1F80008C1F80008698D0008DE
:10816000C1F80008C1F80008C1F80008C1F800080B
:10817000C1F80008C1F80008C1F80008C1F80008FB
:04818000C1F800083A
:1081840010B5054C237833B9044B13B10448AFF34D
:1081940000800123237010BD74050020000000003E
:1081A40030FB00080C4B43B10C480D4910B5AFF33C
:1081B40000800C48036823B910BD0A48036833B92A
:1081C4007047094B002BF7D0BDE810401847064B09
:1081D400002BF5D0184700BF0000000030FB00085A
:1081E40078050020740500200000000010B514205C
:1081F40000F080FC1228074C09D1152000F07AFC0D
:10820400342804D1102000F075FC207010BD082320
:10821400237010BD900500202DE9F041C14DC24FDF
:108224006E78032E88B040F0A2803B784BBBBF4EE3
:10823400737834781C44F37903341C44B3791C44B4
:1082440073791C44337902201C4400F0D5FD0120CD
:1082540000F0D2FD307800F0CFFD707800F0CCFD56
:10826400F07900F0C9FDB07900F0C6FD707900F036
:10827400C3FDE4B2307900F0BFFD204600F0BCFD40
:1082840009E0012B07D1AA4E0024305D013400F02F
:10829400B3FD092CF9D100236B703B70AB7813B19B
:1082A400012000F08BFE0DF1070000F0BFFD044635
:1082B400002800F0D78000F0D5FD08B10023EB7052
:1082C400EA789DF80710531CDBB22A44092BEB70A3
:1082D400117121D12A790023012AEB701CD1954810
:1082E4001A46195C01330A44082BD2B2F9D12B7B0C
:1082F400934240F0B580904B6A791A70AA795A700B
:10830400EA799A702A7A9A716A7A5A71AA7A1A71EF
:10831400EA7ADA7003236B706B7803F0FB02032AAA
:1083240002D0052B40F03581834ADFF800821378B0
:1083340088F80130642188F80010472BD2F8031024
:10834400C8F804104446164600F0328100F2C88092
:10835400422B00F0218100F2B8800A2B00F00C813E
:1083640000F2AB80092B00F0FB80022348E2042ECC
:1083740021D16E4C00234FF001080220637063602A
:1083840084F8008000F038FD404600F035FD207888
:1083940000F032FD607800F02FFDE07900F02CFD54
:1083A400A07900F029FD607900F026FD207900F025
:1083B40023FD304662E7072E33D13B7805A833BB53
:1083C4005A4A137892F801E0D6798DF8163073443E
:1083D400947951798DF819400333334412798DF827
:1083E4001A101C444FF0020C21448DF814C08DF86F
:1083F4001B204FF0010C0A448DF815C08DF817E0CE
:108404008DF818608DF81C2000F062FF43E7012B03
:10841400FAD1474900235A5CC2540133092BFAD1DB
:10842400F2E7082E7FF437AF4049002301224B7056
:108434004B600A708DF8173002218DF818308DF8D2
:1084440019308DF81A308DF81B3004238DF8141070
:108454008DF815208DF816208DF81C3005A8D3E76B
:10846400042358E702AE304600F01EFF00283FF414
:1084740053AF2346F25C01331444082BE4B2F9D120
:108484009DF81020A2427FF446AF2B4B9DF80920A3
:108494001A709DF80A205A709DF80B209A709DF866
:1084A4000C209A719DF80D205A719DF80E201A71B6
:1084B4009DF80F20DA7007232DE7402B67D0412B5E
:1084C4007FF453AF00F01FFA63E0442B6AD066D305
:1084D400452B6AD0462B7FF448AF00F03EFA58E0B3
:1084E400932B00F0118129D88F2B7FD00AD8882BA9
:1084F4007FF43BAF5378012B6DD05CD3052B39D17E
:10850400012342E0902B00F00C81922B7FF42DAFDD
:108514009378002B00F0A380FF2B00F0B38004239A
:108524006EE100BF900500209B060020A8060020F5
:108534009C0600209405002094060020952B00F052
:10854400E980C0F0B280F22B00F05C81FF2B7FF455
:108554000CAF40F2D24399421BD10123AB7018E017
:108564005378013B032B05D8DFE803F01313021300
:1085740001290ED9032343E15378013B032BF9D896
:10858400DFE803F0020202560023636001E000F01A
:10859400B9F908B0BDE8F08100F0CAF9F9E700F0D4
:1085A400D9F9F6E700F0D7F9F3E700F0D5F9F0E7E9
:1085B40000F0D4F9EDE70123BE4A3B7002231370A7
:1085C400BD4B196800230139013311F8010FD05450
:1085D400082BF9D1DDE700220C2188F8072088F860
:1085E400061088F8053088F80420D2E75378042B65
:1085F400C0D8DFE803F0031811111C00142000F0A8
:1086040079FA12280CD1152000F074FA342807D115
:10861400102000F06FFA2870022363712B7810E0A9
:1086240008232B70F8E7F3782B70022208E071B965
:108634002B78082BF9D0A3F11A02012AF5D90622C6
:10864400627123710423E3710023A371A1E7F3781A
:10865400082BE1D01A3B012BDED90623DDE7507845
:10866400831FDBB21E2B00F20C81944A22FA03F31F
:10867400DA0700F10981392800F00681000102F0CF
:108684000FFE86E798F804306B74507898F805303C
:10869400AB7498F80630EB74082298F807308849D0
:1086A4002B75000102F037FE73E793782BB1FF2B93
:1086B40017D0042388F800306BE75078831FDBB2AF
:1086C4001E2B00F2EA807D4A22FA03F3DB0700F155
:1086D400E780392800F0E480000102F0FBFE6060CE
:1086E40057E7507877490822000102F03AFF2B7FC0
:1086F40088F80730EB7E88F80630AB7E88F80530C2
:108704006B7E88F8043044E7D178B2F8010002F0B7
:1087140063FF3EE7B2F8010003F019F8C8F804005B
:1087240037E75578012D3ED032D3022D7FF422AFA6
:108734004FF4A06002F0DFFFC10760D5012140F2D1
:10874400015002F049FF40F2025003F000F8020425
:10875400F9D4D6F8031040F20450091402F090FF43
:10876400D6F803104FF4A16089B202F089FF40F2F9
:10877400025002F0ECFF40F4007140F2025002F0AB
:1087840052FF40F2025002F0E2FF0304F9D431E058
:108794005221412002F020FF4521412002F01CFF1C
:1087A40053214120B3E74FF4A06002F0A4FFC707B0
:1087B40025D5294640F2015002F00EFF40F2025046
:1087C40002F0C5FF0504F9D4D6F8031040F20450B2
:1087D40002F056FF40F2025002F0B9FF40F48071FB
:1087E40040F2025002F01FFF40F2025002F0AFFFCD
:1087F4000004F9D44FF4A16002F0DFFF6FE7062311
:108804002370C6E65378812B7FF489AE9378922B3C
:108814007FF485AE9379A32B7FF481AE5379B42B87
:108824007FF47DAE1379C52B7FF479AED378D62B44
:108834007FF475AE00F064FD00F0D4F9044600F056
:10884400D1F9001B0028B8BF4042B0F57A7FF6DBAF
:1088540072B600F0C1FB1C4B1C4800241C6021466E
:1088640003F0F7FC194803F031FC03F077FA03F046
:10887400B1FD4FF0804004F010FB204600F09EFB59
:1088840087E637287FF4F7AE23796B736379AB738C
:10889400A379EB73E3792B747BE637287FF419AF64
:1088A4002B7EE371EB7DA371AB7D63716B7D2371D3
:1088B4006FE600BF9C060020000000200300005863
:1088C4009D050020A505002010E000E01064024092
:1088D400704710B5094C00F085F92368C01A0028C8
:1088E400B8BF4042FA2807DD054A536983F0010303
:1088F400536100F077F9206010BD00BFB00500207F
:10890400001002407047074B5A78012A05D104220F
:108914000549D3F8030000F00AB9044B03221A7086
:10892400704700BF94060020AC060020A806002073
:10893400064B5A78012A04D19978D3F8030000F041
:108944000FB8034B03221A70704700BF940600202F
:10895400A80600207047704770477047704700BFF3
:1089640038B5012204460D464FF48270062100F00A
:10897400ADFD002205214FF4827000F0A7FD012215
:1089840000214FF4827000F0A1FD8207F1D500228E
:1089940002214FF4827000F099FD0022C4F30721F4
:1089A4004FF4827000F092FD0022E1B24FF4827025
:1089B40000F08CFD012229464FF4827000F086FD00
:1089C400002205214FF4827000F080FD0122002175
:1089D4004FF4827000F07AFDC307F1D438BD2DE95D
:1089E400F843044688461646062101224FF4827055
:1089F40000F06CFD002205214FF4827000F066FD4A
:108A0400012200214FF4827000F060FD8507F1D54A
:108A1400002202214FF4827000F058FD0022C4F3BA
:108A240007214FF4827000F051FD0022E1B24FF4AF
:108A3400827000F04BFD0025771EB5420FD1002255
:108A440005214FF4827000F041FD012200214FF412
:108A5400827000F03BFDC307F1D4BDE8F883013414
:108A640014F03F0918F8051042D0781B42424241E5
:108A74004FF4827000F02AFDB9F1000F36D1BD42E7
:108A840034D2002205214FF4827000F01FFD002132
:108A940001224FF4827000F019FDC107F1D40122C4
:108AA40006214FF4827000F011FD002205214FF4DD
:108AB400827000F00BFD012200214FF4827000F05F
:108AC40005FD8207F1D5002202214FF4827000F0E7
:108AD400FDFC0022C4F307214FF4827000F0F6FC81
:108AE4000022E1B24FF4827000F0F0FC0135A4E7FB
:108AF4000122BDE710B50022044603214FF4827021
:108B040000F0E4FCC4F3072100224FF4827000F06B
:108B1400DDFCE1B200224FF4827000F0D7FC0122A8
:108B240000214FF48270BDE8104000F0CFBCF8B5CE
:108B340004460E461546032100224FF4827000F0CD
:108B4400C5FCC4F3072100224FF4827000F0BEFC80
:108B5400E1B200224FF4827000F0B8FC7719344679
:108B6400013DBC4200D1F8BDA21BAB1A5A425A4186
:108B740000214FF4827000F0A9FC04F8010BF0E727
:108B840068460C4A20F007018D46136801B501338D
:108B94001360094B1A78092A8BBF5A681A78013274
:108BA40001328ABF5A60D2B200221A70BDE8014075
:108BB40085467047B0060020B4050020074B40F2FC
:108BC400DB525A60064AF02182F8231000229A6090
:108BD40007221A606FF0040005F0D6B810E000E038
:108BE40000ED00E0014B5868704700BFB405002059
:108BF40070B5064688B0564804F094FE0121202042
:108C040003F0C0FE0121042003F08CFE02250024A1
:108C1400402302A94F4802938DF80C508DF80E4062
:108C24008DF80D508DF80F4003F0C2FC802302A98B
:108C3400484802938DF80C508DF80E408DF80D5075
:108C44008DF80F4003F0B4FC08220621414803F0DC
:108C540039FD40480822072103F034FD04A804F03C
:108C640013FF0B2E71D8DFE806F0700655585B5ED3
:108C74006164676A6C6E4FF4615304A934480493C9
:108C840004F0A8FE4723002401258DF8043001A830
:108C940006238DF805308DF806408DF8075005F051
:108CA40029F840F2FF312A4804F0EFFF2246282138
:108CB400274804F0CBFF2A4640F22771244804F0E9
:108CC400C5FF2A4640F22661214804F0BFFF2A4628
:108CD40040F225511E4804F0B9FF224640F22441D7
:108CE4001B4804F0B3FF224640F64601184804F03E
:108CF400ADFF224640F66A11154804F0A7FF22464C
:108D04006021134804F0A2FF2946114804F0DDFE57
:108D140008B070BD4FF49643AFE74FF4E143ACE7BE
:108D24004FF41643A9E74FF46143A6E74FF4963393
:108D3400A3E74FF4E133A0E74FF461339DE7064B1B
:108D44009BE7064B99E7064B97E74FF4165394E7D6
:108D5400001401400008024090D0030020A1070045
:108D640040420F0020480388990610B514D51F4BC4
:108D74001A6859680132202A08BF00228A4205D0A5
:108D8400196880881944C0B208721A60184A0A2106
:108D940011609A6A174B1A60134803881A0612D591
:108DA400144B1A687AB9114BDC6A196B8C4216D0D1
:108DB400196B4C1C19441C6391F834108180196B95
:108DC400202900D11A63084803885B0606D540F2BF
:108DD400266104F07EFF054B1A6BDB6A10BD40F27E
:108DE400277104F033FFEEE700140140BC050020B6
:108DF400B8060020B40600200A4AD36A116B013376
:108E0400202B08BF00238B420AD0D16A114481F879
:108E14003400D36240F227710122034804F016BFE4
:108E2400704700BFBC05002000140140094B59687D
:108E34001A6891420CD05A68511C1A445960127A2B
:108E440002705A68202A01D100225A60012070471A
:108E540000207047BC050020014B9862704700BF9A
:108E6400BC050020044B1A7802F0FF0012B1002266
:108E74001A700120704700BFBC06002072B6034B75
:108E840000225A601A6062B6704700BFBC05002019
:108E940010B5441E14F8010F00B910BDFFF7ACFF64
:108EA400F8E700BF2DE9F341434F012108460024B0
:108EB400012503F037FD0226384648F201036946CE
:108EC40000938DF804508DF806408DF805608DF8F8
:108ED400074003F06DFB4FF400433B8338464FF4E7
:108EE4008073694600938DF804608DF806408DF810
:108EF40005608DF8074003F05BFB21464FF48000CA
:108F040003F066FC07F580672946304603F00AFD46
:108F14004FF4C25838466946CDF800808DF80450A5
:108F24008DF806408DF805608DF8074003F040FB8E
:108F3400A7F81880294607F58067042003F0F2FC9F
:108F44003846694600958DF804508DF806408DF832
:108F540005608DF8074003F02BFB3D83294608206C
:108F640003F0E0FC07F500672946102003F0DAFC63
:108F74004FF4407369463846009348F203088DF86D
:108F840004408DF806408DF805608DF8074003F025
:108F94000FFB69463846CDF800808DF804508DF8F3
:108FA40006408DF805608DF8074003F001FBA7F833
:108FB400188002B0BDE8F08100000240034B10B1FC
:108FC400034ADA607047034AFBE700BF00ED00E0A4
:108FD4000400FA050100FA0500224FF0FF31930066
:108FE40003F1604303F561430132082AC3F880109A
:108FF400C3F88011F3D1002304481946C218013381
:10900400F02B82F80013F9D1704700BF00E100E0B3
:1090140070477047704700BF7047704712230B803A
:10902400004870470400002004230B800048704768
:10903400160000200020704700207047094B1A6872
:1090440030B501440024814203D104B11A600020E8
:1090540030BD3F2A04D89C180578257101320124BB
:109064000130F0E71006002010B5044C04480A460D
:10907400214605F03FFB204610BD00BF5F1D0020C8
:10908400E1FA000810B5044C04480A46214605F0EC
:1090940031FB204610BD00BF5F1D0020F3FA00081D
:1090A40010B5044C04480A46214605F023FB20462B
:1090B40010BD00BF5F1D00200BFB000810B5044C61
:1090C40004480A46214605F015FB204610BD00BFA2
:1090D4005F1D002013FB000810B5044C04480A4629
:1090E400214605F007FB204610BD00BF5F1D002090
:1090F4001EFB0008202803D021280BD00020704735
:109104000C4B0A689A610A791A774A795A778A79EC
:109114009A77F3E7074A93690B70180A4870180C9A
:109124001B0ECB70137F0B71537F4B71937F887031
:109134008B71E3E7040000200020704770477047FC
:10914400704770477047F7B5274C4FF4C05300265B
:10915400032700936946022320468DF804308DF8D6
:1091640005708DF806608DF8076003F021FA20463B
:109174000A220B2103F0A6FA0A2220460C2103F04E
:10918400A1FA01254FF400736946204600938DF837
:1091940005708DF804608DF806508DF8076003F0B3
:1091A40007FA0A222046092103F08CFA4FF480635F
:1091B4006946204600938DF806508DF807508DF8C7
:1091C400057003F0F5F90A221146204603F07AFAF5
:1091D40029464FF4804003F0D5FB2946802003F054
:1091E400ADFB03B0F0BD00BF0000024007B54FF473
:1091F400C06004F075FD43238DF80430032201237D
:1092040001A88DF805308DF806208DF8073004F09C
:1092140071FD03B05DF804FB782358430723B0FBCA
:10922400F3F0002301339842FCD270474FF47A7371
:109234005843FFF7F1BF684620F007018D4601B59A
:10924400034806F029F8BDE801408546704700BF91
:10925400C0060020F0B5094B094D014400268842A0
:1092640000D1F0BD1C68621C1A6010F8017B2F55F8
:10927400B2F5006F28BF1E60F1E700BF780600203A
:109284005F150020074B196830B541B100221D1D40
:10929400545D845401329142FAD100221A60084686
:1092A40030BD00BF10060020084B1A68082A10B50C
:1092B4000AD900221C1D115D81540132092AFAD1F8
:1092C40000221A60012010BD002010BD10060020ED
:1092D4000921FFF7BFBF07B5064A074802F13C035F
:1092E40000932032054B012104F078FE03B05DF8B1
:1092F40004FB00BF04000020C00600201801002069
:10930400014805F09DBF00BFC00600202DE9F04FC5
:10931400012189B002256A4FDFF8ACB14FF48050C7
:10932400002403F02FFB38232846012101938DF8F4
:109334000A408DF80B408DF808508DF8095003F061
:10934400F1FA01A9384603F033F9052211463846EB
:1093540003F0B8F938460522042103F0B3F90522D5
:109364003846032103F0AEF901264FF4827A4FF414
:1093740000794FF0200803A95846ADF80C40ADF829
:109384001040ADF81A40ADF81C40ADF80EA0ADF891
:109394001250ADF81460ADF81690ADF8188003F0D3
:1093A400F7FB3146584603F08CFC31464FF48040BD
:1093B40003F0DCFA4FF460433146284601938DF8FC
:1093C4000A408DF80B408DF808508DF8095003F0D1
:1093D400A9FA01A9384603F0EBF8384605220D2115
:1093E40003F070F9384605220E2103F06BF90522CB
:1093F40038460F21A7F5E63703F064F903A9384688
:10940400ADF80C40ADF81040ADF81A40ADF81C4072
:10941400ADF80EA0ADF81250ADF81460ADF816908A
:10942400ADF8188003F0B4FB3146384603F049FC2C
:1094340031464FF4004003F099FA07F5E8374FF44A
:10944400E0533146042001938DF80A408DF80B4017
:109454008DF808508DF8095003F064FA01A93846D4
:1094640003F0A6F8384606220A2103F02BF9384601
:1094740006220B2103F026F9062238460C2103F0BC
:1094840021F9ADF80C40ADF81040ADF81A40ADF834
:109494001C400C4CADF80EA003A92046ADF81250A8
:1094A400ADF81460ADF81690ADF8188003F070FBB9
:1094B4003146204603F005FC09B0BDE8F08F00BF3B
:1094C40000040240003C004000300140B0F5827FBF
:1094D400F8B504460E46154650D040F20123984292
:1094E4002FD040F2011398425BD12F4B4FF400422E
:1094F4002E4F5A830221384603F071FC0028F9D01C
:1095040031462A48294E03F037FC0121304603F046
:1095140066FC0028F9D0002D36D0B4F5827F30D017
:1095240040F201239C4223D040F201139C4238D1E3
:109534001D4B4FF400421A831C4803F01AFCC5B2B9
:109544002DE01B4B1B4C4FF400425A830221204652
:1095540003F045FC0028F9D031461648154C03F0B9
:109564000BFC0121204603F03AFC0028F9D01DB180
:109574000F4B4FF400421A830E48DEE701220E4BD4
:10958400B6E701220C4BD6E7B4F5827FD4D040F283
:1095940001239C42F0D040F201139C42CCD02846D7
:1095A400F8BD0025FBE700BF00000240003C00407E
:1095B4000010024000380040000802407047FEE7F7
:1095C400FEE7FEE7FEE7704770477047704700000C
:1095D4002E4B1A68002142F001021A6099601A6841
:1095E40022F0847222F480321A60294A5A601A687E
:1095F40082B022F480221A60D960009101911A6825
:1096040042F480321A6019461A6802F40032019258
:10961400009A01320092019A1AB9009AB2F5A06F29
:10962400F2D10B6813F4003318BF01230193019B9B
:10963400012B04D0174B184A9A6002B07047134BA1
:109644009A689A609A6842F400429A609A6842F46E
:10965400A0529A60114A5A601A6842F080721A60E5
:109664001A689201FCD50E4A40F2037111609A689F
:1096740022F003029A609A6842F002029A60034A56
:10968400936803F00C03082BFAD1D3E700380240A7
:109694001030002400ED00E000800008081E4005A2
:1096A400003C0240144A15499068154B00F00C0028
:1096B400042810B501D008280AD00B600E4B9B6813
:1096C400C3F303130B441A790B68D3400B6010BD2A
:1096D400546850685268C2F3881200F03F00B3FB2C
:1096E400F0F35343044A5268C2F301420132520078
:1096F400B3FBF2F3E1E700BF003802407C00002036
:109704000024F400704770470020704710B5064CE1
:10971400204602F00DFB054B1A88054B204619889C
:10972400BDE8104001F0AEBBFC0C00206C0D002025
:10973400800D002010B5064B064C1A88064B2046B7
:10974400198801F037FB2046BDE8104002F0F6BA54
:109754005E0D0020B60C0020640D002070B4534B45
:1097640053481B78534943B10123037000230B7002
:109774000978007870BC01F021BC4F4B1A88013283
:1097840092B2322A1A8005D0642A03D0962A01D0D4
:10979400C82AEDD1494C2578494C05F00F05013D07
:1097A400072D45D8DFE805F04404423E44444440D4
:1097B400402525702578AC0601D4C82A12D115F0AD
:1097C4001F0218BF52009C781CBF02F1FF32D2B2B4
:1097D400AC422FD02E064CBF00220122027001227F
:1097E4009A809D70374A1578AA0602D41A88C82A26
:1097F40012D115F01F0218BF52009C791CBF02F150
:10980400FF32D2B2AC4233D02E064CBF002201222A
:109814000A7001221A819D711A88C82A04BF002285
:109824001A80A5E74125C4E70125C2E76025C0E702
:109834000025BEE76C0617D50478B4FA84F46409ED
:109844000470002ACDD09C880134A4B294429C8038
:10985400C7D92E0602F104024CBF01260026A242FB
:109864000670BEDA0022BBE705F001020270B8E719
:109874006C0617D50C78B4FA84F464090C70002AC9
:10988400C9D01C890134A4B294421C81C3D92E06C8
:1098940002F104024CBF01260026A2420E70BADA7D
:1098A4000022B7E705F001020A70B4E7760D002044
:1098B400400D0020FA0C0020540600205D0D00200D
:1098C400660D00207E0D0020064B1B783BB1064A36
:1098D400B2F90030002BC4BF03F1FF331380FFF74C
:1098E4003DBF00BF6A0D0020720D002037B502ACE9
:1098F400002501F065F844F8045D042220464FF485
:10990400A06101F01EFA019B204623F47F43042248
:109914004FF4A061019301F084FA034B012228461D
:109924009A7203B030BD00BF5406002008B51C4B2A
:109934009B7A002B32D01B4B1B7883B11A4B1B78BC
:10994400CBB101F079FB092803D9FFF7BDFF01F082
:1099540079FB01F091F8BDE8084000F073BF01F015
:10996400C0FA420510D5104B01221A700F4B1B7818
:109974000BB1FFF7DFFE02F0E7F90D4B1B78002B6C
:10998400DFD0FFF7C3FEDCE70A4B1B88002BF2D1C4
:10999400030542BF044B01221A70ECE708BD00BF67
:1099A400540600207B0D0020700D0020760D002051
:1099B4007A0D00205E0D002002F0C6B92DE9F04FAB
:1099C40085B0884601904FF4A06103A89246022214
:1099D400994601F0B6F9022240F202510DF10E004F
:1099E40001F0AFF9BDF80C4014F0010400F08480DC
:1099F400B9F1000F06D1BDF80E3013F0400F14BFBB
:109A0400042402244FF4807302224FF4A06103A8BB
:109A1400ADF80C3001F005FA00264FEA440B0A2792
:109A2400354645450DD30024002303A802224FF4F4
:109A3400A061ADF80C3001F0F4F9204605B0BDE8A2
:109A4400F08F042240F204510DEB020001F0E9F919
:109A5400B9F1000F34D14FF48073022240F2025165
:109A64000DF10E00ADF80E3001F0DBF9022240F2E8
:109A740002510DF10E0001F064F9BDF90E30002B16
:109A8400F4DB022240F202510DF10E0001F059F90B
:109A9400BDF80E3013F4F04F1CD09B0400D46FBB00
:109AA400013FFFB2BDF80E3003F4F0432BB9019B24
:109AB400264423440193B6B20A272544ADB2B0E745
:109AC40002224FF4A1610AEB450001F0AAF94FF418
:109AD4000073C2E7B9F1000FE4D133194345C3BFA2
:109AE400A8EB0602520092B25A464FF4A1610AEB67
:109AF400450001F026F9D5E7502495E7512493E772
:109B040010B586B0FF23ADF8063002AC0023224620
:109B140007211846FFF752FF00BBBDF80630225C50
:109B24005340082213F0800F02F1FF324FEA43033F
:109B340018BF83F0070392B29BB2002AF2D101301E
:109B44000E28ECD106AADBB222F8123D01231946F5
:109B54000720FFF733FF002808BF202006B010BD00
:109B6400034A00231380034A1360034A13607047B7
:109B7400480D00204C0D0020500D002001880729BD
:109B840038B5044640F2F88003890839013B89B2AC
:109B9400052B00F2B680DFE803F00345566C8D9781
:109BA4007A4B1D88002D40F0EC8000F11002C36850
:109BB400104600F0EBFF764B01221A60754B1D60D6
:109BC400754B186047F69573984200F28B80704B82
:109BD4001B68E36000F108032380704B1B880E3B75
:109BE40003229842694B22810CBF012204221A806D
:109BF4006B4B1D78002D00F0B7806A4B62791978A1
:109C0400490704BF01211970197802F00F0262712B
:109C140042EA0112627101312046197001F002FF1B
:109C2400002038BD594B1D88002D40F0AA80C26821
:109C3400103000F0DDFF47F6FD73002808BF18461A
:109C4400534B1D60BEE7514B1B8823F004039BB2AA
:109C5400022B40F096804E4BC2681B689A4240F03B
:109C64008D80103001F002F80028ABD147F6FD706A
:109C74004FE0464B1B88012B0FD1474D00F11001DB
:109C8400286801F025F8434A2B681360404A0344CE
:109C94002B6013680133136094E747F6FE7048F2B3
:109CA4000402042B18BF1046050442D4374B00208D
:109CB400188038BD354B1B88002B62D0C06801F07A
:109CC4002BF847F6FF70EFE7304B1B88012B01D0D0
:109CD400042B56D12F4BA089196804F1100201F00E
:109CE40017F86FE747F6FA7398420CD806232381D6
:109CF400A0F5FF4000237A38E3810823A081238064
:109D040076E748F20400A0F5FF437C3B9BB2012BAD
:109D1400CAD81F4A1368E360591C082311602380C2
:109D240047F6FD730422984222811BD10222174B6D
:109D34005DE70523238108232380E060002303F0EB
:109D4400FE022244128A12F0FF0F04D012F47F4F55
:109D540004D10133DBB20933238003E00233DBB2E5
:109D6400202BECD10022E2E74021204601F014FF31
:109D740050B10D4B1C6053E7062038BD48F2050076
:109D840092E748F204008FE738BD00BF480D002079
:109D94004C0D0020540D0020440D0020B41400206C
:109DA400740D0020A8140020500D002010B5044CA0
:109DB400206820B1002101F0EFFE0023236010BDD4
:109DC400500D00205C4B1B88B3F5405F73B505460E
:109DD400C0F0B080002001F021F98379DE0701D4BE
:109DE4001624A4E0037903F00C02042AF8D19C079A
:109DF400F6D54388223B9BB2DE2BF1D80388A3F52A
:109E040080539BB2B3F5005FEAD8012001F006F954
:109E14008379DB07E4D5037913F00C04E0D19907C7
:109E2400DED54388223B9BB2DE2BD9D80388A3F529
:109E340080539BB2B3F5005FD2D8032D26D93F4E91
:109E440001230320337001F0E9F882794388D207B3
:109E540040D59BB13A4A12889A420FD1442A0DD870
:109E6400027912F00C0F09D13649038809780229C6
:109E740006D1A3F58053B3F5005F05D91E2456E03F
:109E8400314909889942F9D1900720D4022D37D954
:109E9400022001F0C3F882794388D10735D5A3B1F4
:109EA4002A4A12889A4210D1442A0ED8037903F020
:109EB4000C02042A09D1234902880978022910D105
:109EC400A2F58052B2F5005F0FD91D242FE00023C4
:109ED4003370DDE7002BD1D1194B1B88002BCDD17A
:109EE400D4E71B4909889142EFD113F04001194A84
:109EF40018BF012111709A0702D5104B00221A7065
:109F040000238DF80730144E0EE0002BDDD10F4BEB
:109F14001B88002BD9D1F3E7284601F07FF80135DF
:109F240083798DF80730EDB23378AB42F4D820460C
:109F340002B070BD1424FAE76E0D0020580D002005
:109F44006C0D00205D0D0020800D00205E0D0020B2
:109F5400640D00207C0D00207D0D00202DE9F341CF
:109F64005F4A604E604C614D002302201370ADF8CF
:109F74000430ADF80630338001F050F803882380B4
:109F84000379032013F0020F0CBF4FF003084FF0C6
:109F9400010801F043F8564A038813800279B5F8A2
:109FA40000E012F0020F534A0CBF0321012117886D
:109FB4000EFB0131B94205DD4F4A12883A449342FF
:109FC400C0F285804D4A1088814204DD4C4A1188D4
:109FD40001448B427BDB21884A4C228808FB021215
:109FE400974206DADFF810C1BCF800C06744B942F2
:109FF4006FDB904204DA424F3F883844814268DB89
:10A00400934202DA7344994263DB012240F68111E0
:10A014000DF1030000F095FE9DF8033013F0090FD5
:10A0240059D1394B1B78002B57D0384B1B782BB1A7
:10A034002388002B3AD04FF48063338002224FF4FC
:10A0440084610DF1060000F07CFE2388304E002B65
:10A0540035D0BDF8063093B302224FF4806101A8D5
:10A0640000F06FFEBDF8043033B3BDF806200233B0
:10A0740046F2A71103FB021346F2A812B3FBF2F354
:10A0840033803288234B1B78EAB9F3B9238813B1A0
:10A09400022000F0ABFF2B8813B1032000F0A6FFD1
:10A0A400FFF734FB002002B0BDE8F0812B88002BC1
:10A0B400C4D04FF40063C0E7ADF80630E0E70023F6
:10A0C400ADF80430DCE7002BE0D11F20EBE71E20C5
:10A0D400E9E71D20E7E73020E5E72920E3E700BFB3
:10A0E400700D0020680D0020640D00206C0D002010
:10A0F400800D0020BE140020B4140020AC140020F5
:10A10400C61400205E0D0020580D00207B0D002099
:10A11400780D00207C0D0020024B187808B1024B0A
:10A1240018887047620D0020600D0020024A002349
:10A134001370024A13707047700D0020760D0020D2
:10A1440008B50B4B1B8813B1022000F038FF094BF4
:10A154001B8813B1032000F032FF074A0023137059
:10A16400064A1370064A1370064A137008BD00BFEE
:10A174005E0D00206C0D0020700D00207C0D002071
:10A184007A0D00205F06002073B51C4DADF8061053
:10A194002B7883424FF6FF7318BF28709942064606
:10A1A4000C4606D002224FF49A710DF1060000F01D
:10A1B40038FE2B78ADF8063002224FF498710DF179
:10A1C400060000F02EFE0E4A0CB1F10603D4002363
:10A1D400137002B070BDA4F11A0399B218299DBF7F
:10A1E400084BCB40DB430123DB0701D44123EFE7DA
:10A1F4001B2C0CBF42234023EAE700BF5D0D002067
:10A204007E0D0020010008012DE9F04FC34FC44D1D
:10A21400C44C85B04FF6FF733B80012210F010034D
:10A22400029301912A7000F00F00237833D023F0B9
:10A234001003237002922378DFF80883C6B206EB7A
:10A24400031303F0FF0BBBF1440F3AD032D8BBF138
:10A25400220F3FD028D8BBF1120F3BD0B249039153
:10A264004FF0000ABBF1310FA1F800A000F02881E3
:10A2740000F2A580BBF1180F58D000F28F80BBF11B
:10A28400120F00F036814AD8BBF1110F00F08F8114
:10A294004FF012094CE0DA0602D5012840F00D8196
:10A2A40003F00F032370C6E7BBF1240F1BD0BBF1EF
:10A2B400420FD2E7BBF1820F0CD005D8BBF1480F97
:10A2C400CCD19A4A107806E0BBF1840FF9D0BBF1E7
:10A2D400880FF5E70220FFF775FD1FFA80F9B9F141
:10A2E400000F07D1BAE79249924801F01CFD81465C
:10A2F4000028E6D02278042A00F07881082A00F0A9
:10A304007181022A40F07981B9F1160F40F073810E
:10A3140001F026FB01F0FDFC0123237008E0BBF1F2
:10A32400130F00F09680BBF1140FB1D14FF0110957
:10A33400207800F00F039E4200F08981B9F1000FEC
:10A3440003D1019B002B00F07E81304303070ED51F
:10A35400794B1B781BB101F0E4FCFFF7E7FE744B6B
:10A364001B88002B00F06481022000F028FEB9F164
:10A37400000F00F064812378082B04BF04232370AA
:10A38400237843F0100323700023207888F80030EA
:10A39400494605B0BDE8F04FFFF7F6BEBBF1230F09
:10A3A400C4D005D8BBF1210F21D0BBF1220F6DE73A
:10A3B400BBF1240F00F0C880BBF1280FB5E7BBF157
:10A3C400480F00F0D28020D8BBF1420F32D016D80B
:10A3D400BBF1410F7FF45CAF01F09FFC8146FFF7B6
:10A3E400AFFE00232B70B9F1000F40F05D8101F046
:10A3F400B7FA01F08EFC4FF0210B81466EE0BBF101
:10A40400430F93D0BBF1440F40E7BBF1830F8DD0D2
:10A4140018D8BBF1810F00F0C080BBF1820F7FF42C
:10A4240037AF01F07EFC8146FFF780FE85F800A07F
:10A43400002853D101F071FCFFF782FE002129703E
:10A44400894675E7BBF1840F00F09F80BBF1880F4C
:10A454001CE7DFF8ECB0012302208BF80030FFF793
:10A46400B1FC20B18BF800A04FF0150960E701F0B2
:10A4740049FA1FFA80F9B9F1000F40F0EC8085F831
:10A48400009001F044FC8146002840F0E4802B4B0E
:10A4940001221A700320FFF735F9B9F1FF0F7FF499
:10A4A40047AF0123039A88F80030132313804FF435
:10A4B400FA633B803B88323B3B8005B0BDE8F08FBC
:10A4C4001F4801780029BBD080F800A00220FFF7C4
:10A4D40079FC01F045FA01F01CFC8146B9F1FF0F4B
:10A4E4007FF426AF039B012288F80020A3F800B074
:10A4F40096E001F007FA1FFA80F9B9F1000F40F075
:10A50400B58085F8009001F002FC8146002840F0F7
:10A51400AD800A4B01221A700AE700BF720D0020B9
:10A524005C0D00205D0D00205A0D00207D0D0020E3
:10A534005E0D00206C0D0020760D0020AA14002072
:10A54400740D00206A0D0020FFF708FD81460028E5
:10A5540040F096802870564801F0DDFB81460028C3
:10A5640040F08E800122534BD5E7FFF7D5FD81469D
:10A57400002840F08F80287001F0D1FB814600282C
:10A5840040F0888001224C4BC5E701F0CAFBD1465C
:10A59400FFF7CCFD85F800A0CAE601F0C2FB8146B6
:10A5A400FFF7C4FD85F800A0002897D114E7029BAB
:10A5B40013B1584601F0AAFB404B1B784BB92378E2
:10A5C40013F00C0F05D03E4B1B882BB1022000F07A
:10A5D4000DFD4FF0FE09ABE63A4B1B88002BF8D07B
:10A5E4000320F4E701F09DFBFFF7A0FD01F095FBCC
:10A5F400FFF7A6FD88E602222270B9F1FF0F7FF46F
:10A6040097AE012288F800202F4ABBF1240FA2F84C
:10A6140000B00AD006D8ABF11203012B7FF647AF86
:10A62400C82346E7BBF1480FFAD142F2283340E78A
:10A63400244B1B88002B3FF49AAE032095E6019B24
:10A644000BB146F010062670DDF804909CE600215C
:10A6540088F800109DE6B9F1FF0F3FF41BAF2B788B
:10A664000BB901F056FB01F07BF913E7B9F1FF0FC9
:10A67400C7D02B780BB901F04CFB01F071F957E608
:10A68400B9F1FF0FBDD02B780BB901F046FBFFF7F2
:10A6940057FD4DE6B9F1FF0FB3D02B780BB901F09C
:10A6A40040FBFFF743FD43E64FF0410B16E700BFC5
:10A6B400680D00207A0D0020760D0020620D002028
:10A6C4005E0D00206C0D00205A0D002038B5514D50
:10A6D4002B788BB1504B514CB3F90030002B3BD14C
:10A6E4002388242BC3F307142ED006D8123B012B46
:10A6F40010D9002C40F08A8038BD482BF9D1484B42
:10A704001B780BB901F00DFBFFF710FD1B20002C8B
:10A7140077D138BD424B1B780BB901F0FAFA01F03E
:10A724001FF9404B1B78002B6ED03F4B1888002C30
:10A73400E2D000232B7008B144F0100401462046F7
:10A74400BDE83840FFF720BD354B1B780BB901F04D
:10A75400E4FAFFF7F5FCE4E72388242B1FD003D8A1
:10A76400123B012B03D938BD482B2FD038BD2C4BBD
:10A774001A78002AC0D000221A7001F0C8FA30B941
:10A784002A4B247801221A7004F00F04B1E7FF2841
:10A79400B2D001F0BEFABDE8384001F0E1B8204B78
:10A7A4001A78002AA8D0002221481A7001F0B3FABE
:10A7B40020B9204B01221A700424BAE7FF289BD049
:10A7C40001F0ABFABDE83840FFF7BABC144B1B7874
:10A7D400002B91D0184B1B881BB1184B1B78002BF6
:10A7E4008AD001F09CFA20B9154B01221A70082472
:10A7F4009FE7FF2880D001F094FABDE83840FFF7C6
:10A8040095BC00232B7097E7012080E70020287077
:10A8140094E700BF6A0D0020720D00205A0D00203D
:10A824005C0D0020620D0020600D0020AA140020A1
:10A83400680D00207A0D00205E0D0020700D0020B0
:10A84400760D00200E4B1B8807B59BB102A8002390
:10A8540020F8023D02224FF4886100F072FABDF83C
:10A864000630DB0706D4074B1B7833B11B210420C9
:10A87400FFF7CAFC03B05DF804FB034A1370F9E761
:10A88400780D0020760D0020700D002070B5404D2D
:10A894002B780C46002B50D03E4B1B7853B100292B
:10A8A4006FD03D4B01221A703C4B19803C4B002267
:10A8B4001A8070BD3B4E49B3374B01221A70374B97
:10A8C40019803388242B1CD00FD8123B934213D900
:10A8D4003088C0F3071000232B700CB140F0100037
:10A8E4002146BDE87040FFF74FBC482BF0D101F082
:10A8F40018FAFFF71BFCEBE701F00BFA01F030F854
:10A90400E6E701F00AFAFFF71BFCE1E730882428A8
:10A9140010D006D8A0F11203012B07D900F00F00C4
:10A92400D9E74828FAD101221F4B01E01F4B01222D
:10A934001A70F3E701221E4BFAE7174D79B1012390
:10A944002B70164B19801B4B1B7800F00F0203F081
:10A954000F039A4215DABDE87040FFF755BC2B7817
:10A964007BB1144B1B7803F00F030C2B05D1124B56
:10A974001B883BB1022000F039FB084A00232B70EE
:10A98400138070BD0D4B1B88002BF6D00320F2E71B
:10A994006A0D00205C0D0020620D0020600D002077
:10A9A400720D00205A0D0020760D0020AA140020FC
:10A9B4007A0D00205D0D00205E0D00206C0D00203E
:10A9C40038B51E4C1E481E4D0122052100F0B9F970
:10A9D40020460222062100F0B4F923889B0203F5E5
:10A9E4008053238000242B78E0B2834204F10104D5
:10A9F40021D800F029FF134B00241C70124B1C704B
:10AA0400124B1C70124B1C70124B1C70124B1C709E
:10AA1400124B1C80124B1C70124B1C80124B1C805E
:10AA2400124B012021461870FFF7AEFB104B1C801F
:10AA3400104B1C7038BD00F0C2FAD4E76E0D002034
:10AA44007D0D00205C0D00206A0D0020700D00209B
:10AA5400760D00207A0D00207C0D0020780D00205A
:10AA6400620D0020600D0020680D00205D0D0020A7
:10AA74005A0D00207E0D0020F7B53E4F002301241F
:10AA8400ADF806308DF8054001F038F93A7832B166
:10AA9400224640F60E010DF1050000F052F900F0D7
:10AAA40020FA10F0010F0446334D10D02E7876B9F9
:10AAB4004FF490710DF10600012200F042F924F0E8
:10AAC400110431469DF80600A4B2FFF79DFBE10690
:10AAD40011D52B787BB9294B187810F010010AD1C5
:10AAE40020F01003012B06D024F0100400F00F0016
:10AAF400A4B2FFF789FB2B780BB1FFF7E7FD3B7896
:10AB040023B39DF8051011F0010105D11B4B1878F2
:10AB140000F00F00FFF778FBA20509D518480023C1
:10AB24000370184B0122198800F07BF900F0DAFF5A
:10AB34009DF8053013F0020F134B1B7808D04BB16E
:10AB440000F0CFF9C30501D501F088F803B0F0BDDA
:10AB5400002BF5D000F0F8FF9DF8053002A803F0B3
:10AB6400020300F8033D012240F60F0100F059F9F9
:10AB7400E6E700BFAA1400206A0D00205D0D002046
:10AB8400670D0020BE140020C814002030B585B025
:10AB94000C4615460A460146684604F0D3FD1049A2
:10ABA40000239AB2944210D80E4B0F4A1B881468A3
:10ABB4000E490E3BA34294BF9CB2A4B2224628463F
:10ABC40004F0C0FD204605B030BD1DF8032001335C
:10ABD400581810F8010C9042E3D048F20104F1E750
:10ABE4008C120020B414002088120020880D00204C
:10ABF400072970B503460D46184915D9048844F24F
:10AC04004530844210D15C8845F2414084420BD1E6
:10AC14009C8845F24670844206D10B78A3B1104655
:10AC2400FEF771FD002070BD0C7884B90F2D11D88A
:10AC34000B4E19462A46304604F084FD094BAC55A8
:10AC44001C60094B1C60EDE748F2080070BD48F237
:10AC5400090070BD48F2030070BD00BF740D0020F0
:10AC64008C120020840D002088120020F8B5134BAC
:10AC74001B780D461BB1BDE8F840FEF745BD104CEE
:10AC84002368CE18B6F5A06F15D829B10A46014637
:10AC94000C48184404F056FD0B4B1B880E3B9D4298
:10ACA40014BF0A4B26604FF000001EBF20601E60D8
:10ACB40047F6FC70F8BD48F20300F8BD740D00209F
:10ACC400840D0020880D0020C61400208812002066
:10ACD40038B50C4B1B6883420D460ED90A4A0B4902
:10ACE40014881B1A0E3C9C4228BF1C460144224671
:10ACF400284604F027FDA0B238BD14BF48F2040072
:10AD0400002038BD88120020B4140020880D0020D3
:10AD140008461146FFF7DCBF10B5064C236843B163
:10AD240010220021044804F0F7FD044A00232360A4
:10AD3400136010BD840D00208C12002088120020A6
:10AD44007047F8B506460C46154672B60022C1F3A4
:10AD5400471140F20110FEF7B9FBE10041F0060192
:10AD6400002201F0FE0140F20110FEF7AFFB210AC0
:10AD740021F01F01002241F00C0140F20110FEF706
:10AD8400A5FB0022FF2140F20110FEF79FFB0024E7
:10AD94006F1EAC4201D362B6F8BDBC4234BF002280
:10ADA40001225142C9B240F20110FEF78FFB305527
:10ADB4000134EEE7F8B50C461546C1F347110022FD
:10ADC400064640F20110FEF781FBE10041F0060166
:10ADD400002201F0FE0140F20110FEF777FB210A88
:10ADE40021F01F01002241F00C0140F20110FEF796
:10ADF4006DFB0022FF2140F20110FEF767FB0024E7
:10AE04006F1EAC4200D3F8BDBC4234BF0022012205
:10AE14005142C9B240F20110FEF758FB30550134DB
:10AE2400EFE7F8B506460C46154672B60022C1F3A4
:10AE3400471140F20110FEF749FBE10041F0060121
:10AE4400002201F0FE0140F20110FEF73FFB210A4F
:10AE540021F01F01002241F0100140F20110FEF721
:10AE640035FB00246F1EAC4201D362B6F8BDBC4270
:10AE7400315D34BF0022012240F20110FEF726FBAF
:10AE84000134F0E7F8B50C461546C1F3471100222A
:10AE9400064640F20110FEF719FBE10041F00601FD
:10AEA400002201F0FE0140F20110FEF70FFB210A1F
:10AEB40021F01F01002241F0100140F20110FEF7C1
:10AEC40005FB00246F1EAC4200D3F8BDBC42315DCB
:10AED40034BF0022012240F20110FEF7F7FA0134D8
:10AEE400F1E738B572B60022114640F20110FEF7C0
:10AEF400EDFA00220446022140F20110FEF7E6FAC0
:10AF040001220546FF2140F20110FEF7DFFA62B686
:10AF140044EA052080B238BD002210B5114640F243
:10AF24000110FEF7D3FA01220446002140F2011079
:10AF3400FEF7CCFA44EA002080B210BD13B5022219
:10AF440004464FF401710DF10600FFF7FAFEBDF857
:10AF540006300DF106001C4002224FF40171ADF8D9
:10AF64000640FFF75EFF02224FF401710248FFF72B
:10AF7400E8FE02B010BD00BFA412002013B50222E7
:10AF840004464FF401710DF10600FFF7DAFEBDF837
:10AF940006300DF106001C4302224FF40171ADF896
:10AFA4000640FFF73EFF02224FF401710248FFF70B
:10AFB400C8FE02B010BD00BFA4120020704737B510
:10AFC40002AC0122C00004F8012D00F60705294651
:10AFD4002046FFF726FF012229462046FFF7B1FE4F
:10AFE4009DF80730DB07F6D503B030BD37B502ACAA
:10AFF4000023C00004F8013D00F60705012229469C
:10B004002046FFF70EFF012229462046FFF799FE4E
:10B014009DF80730DB07F6D403B030BD10B5054CFE
:10B02400C1000822204601F50061FFF78AFE204690
:10B0340010BD00BF9C120020014B1868704700BF70
:10B04400B0060020014B00221A607047B0060020B1
:10B05400F8B504460D46164672B60022C0F34711F1
:10B0640040F20120FEF732FAE10041F0060100222D
:10B0740001F0FE0140F20120FEF728FA210A21F036
:10B084001F01002241F00C0140F20120FEF71EFADC
:10B094000022FF2140F20120FEF718FA7719344606
:10B0A400013DBC4201D162B6F8BDA21B95428CBFE2
:10B0B400002201225142C9B240F20120FEF706FAF1
:10B0C40004F8010BEDE7F8B504460D46164672B6D2
:10B0D4000022C0F3471140F20120FEF7F7F9E10026
:10B0E40041F00601002201F0FE0140F20120FEF7CA
:10B0F400EDF9210A21F01F01002241F0100140F274
:10B104000120FEF7E3F900246F1EAC4201D162B6C0
:10B11400F8BDBC42315D34BF0022012240F201205F
:10B12400FEF7D4F90134F0E7F8B504460D461646A7
:10B13400C0F34711002240F20120FEF7C7F9E100F5
:10B1440041F00601002201F0FE0140F20120FEF769
:10B15400BDF9210A21F01F01002241F00C0140F247
:10B164000120FEF7B3F90022FF2140F20120FEF78F
:10B17400ADF977193446013DBC4200D1F8BDA21B9C
:10B1840095428CBF002201225142C9B240F20120F3
:10B19400FEF79CF904F8010BEEE7F8B504460D46FA
:10B1A4001646C0F34711002240F20120FEF78EF943
:10B1B400E10041F00601002201F0FE0140F201200D
:10B1C400FEF784F9210A21F01F01002241F0100149
:10B1D40040F20120FEF77AF900246F1EAC4200D140
:10B1E400F8BDBC42315D34BF0022012240F201208F
:10B1F400FEF76CF90134F1E738B504460D4672B632
:10B204000022C0F3471140F20120FEF75FF9E1008C
:10B2140041F00601002201F0FE0140F20120FEF798
:10B2240055F9210A21F01F01002241F0100140F2DA
:10B234000120FEF74BF90122294640F20120FEF7D6
:10B2440045F962B638BD38B504460D4672B60022DB
:10B25400C0F3471140F20120FEF738F9E10041F054
:10B264000601002201F0FE0140F20120FEF72EF952
:10B27400210A21F01F01002241F0100140F20120B7
:10B28400FEF724F9E9B2002240F20120FEF71EF98C
:10B294000122290A40F20120FEF718F962B638BDEE
:10B2A40038B504460D4672B60022C0F3471140F289
:10B2B4000120FEF70BF9E10041F00601002201F044
:10B2C400FE0140F20120FEF701F9210A21F01F01DD
:10B2D400002241F0100140F20120FEF7F7F8E9B234
:10B2E400002240F20120FEF7F1F8C5F30721002205
:10B2F40040F20120FEF7EAF8C5F30741002240F2CC
:10B304000120FEF7E3F80122290E40F20120FEF7A6
:10B31400DDF862B638BDF8B504460E46154672B679
:10B324000022C0F3471140F20120FEF7CFF8E100FC
:10B3340041F00601002201F0FE0140F20120FEF777
:10B34400C5F8210A21F01F01002241F0100140F24A
:10B354000120FEF7BBF800246F1EAC4201D162B697
:10B36400F8BDBC42315D34BF0022012240F201200D
:10B37400FEF7ACF80134F0E710B5044672B60022CB
:10B38400C0F3471140F20120FEF7A0F8E10041F0BC
:10B394000601002201F0FE0140F20120FEF796F8BA
:10B3A400210A21F01F01002241F00C0140F201208A
:10B3B400FEF78CF80022FF2140F20120FEF786F808
:10B3C4000122FF2140F20120FEF780F862B610BD91
:10B3D40037B5244C80236383FDF704FC0546FDF751
:10B3E40001FC401B0028B8BF40420428F7DD80233D
:10B3F4002383FDF7F7FB1B4C05462369DB0623D5A6
:10B404000024FDF7EFFB0546FDF7ECFB401B00288D
:10B41400B8BF4042B0F5FA7F21DC02224FF4A0719C
:10B424000DF10600FFF78DFC9DF80630052BEBD1DE
:10B434004FF43070FFF7A0FF09214FF43070FFF78D
:10B44400DBFE204603B030BDFDF7CCFB401B0028DB
:10B45400B8BF4042B0F5FA7FCFDD0124D1E7012423
:10B46400E6E700BF000C024010B5044672B60022A5
:10B47400C0F3471140F20120FEF728F8E10041F043
:10B484000601002201F0FE0140F20120FEF71EF841
:10B49400210A21F01F01002241F00C0140F2012099
:10B4A400FEF714F80022FF2140F20120FEF70EF807
:10B4B4000022114640F20120FEF708F8012204465A
:10B4C400FF2140F20120FEF701F862B644EA0020B1
:10B4D40080B210BD70B5044672B60022C0F34711A5
:10B4E40040F20120FDF7F2FFE10041F006010022E5
:10B4F40001F0FE0140F20120FDF7E8FF210A21F0EE
:10B504001F01002241F00C0140F20120FDF7DEFF93
:10B514000022FF2140F20120FDF7D8FF002211464E
:10B5240040F20120FDF7D2FF00221146064640F208
:10B534000120FDF7CBFF00221146054640F2012011
:10B54400FDF7C4FF01220446FF2140F20120FDF76C
:10B55400BDFF62B6240444EA0060304340EA05209B
:10B5640070BDF8B504460E46154672B60022C0F307
:10B57400471140F20120FDF7A9FFE10041F0060167
:10B58400002201F0FE0140F20120FDF79FFF210A95
:10B5940021F01F01002241F00C0140F20120FDF7CF
:10B5A40095FF0022FF2140F20120FDF78FFF77195C
:10B5B4003446013DBC4201D162B6F8BDA21B95429E
:10B5C4008CBF002201225142C9B240F20120FDF792
:10B5D4007DFF04F8010BEDE738B504460D4672B65D
:10B5E4000022C0F3471140F20110FDF76FFFE100A4
:10B5F40041F00601002201F0FE0140F20110FDF7C6
:10B6040065FF210A21F01F01002241F0100140F2E0
:10B614000110FDF75BFF0122294640F20110FDF7FE
:10B6240055FF62B638BD38B504460D4672B60022E1
:10B63400C0F3471140F20110FDF748FFE10041F06B
:10B644000601002201F0FE0140F20110FDF73EFF69
:10B65400210A21F01F01002241F0100140F20110E3
:10B66400FDF734FFE9B2002240F20110FDF72EFF8E
:10B674000122290A40F20110FDF728FF62B638BD05
:10B6840038B504460D4672B60022C0F3471140F2A5
:10B694000110FDF71BFFE10041F00601002201F05B
:10B6A400FE0140F20110FDF711FF210A21F01F01F4
:10B6B400002241F0100140F20110FDF707FFE9B24A
:10B6C400002240F20110FDF701FFC5F3072100221B
:10B6D40040F20110FDF7FAFEC5F30741002240F2E3
:10B6E4000110FDF7F3FE0122290E40F20110FDF7CF
:10B6F400EDFE62B638BD10B5044672B60022C0F342
:10B70400471140F20110FDF7E1FEE10041F00601AE
:10B71400002201F0FE0140F20110FDF7D7FE210ADC
:10B7240021F01F01002241F00C0140F20110FDF74D
:10B73400CDFE0022FF2140F20110FDF7C7FE0122D9
:10B74400FF2140F20110FDF7C1FE62B610BD10B535
:10B75400044672B60022C0F3471140F20110FDF70F
:10B76400B5FEE10041F00601002201F0FE0140F2C5
:10B774000110FDF7ABFE210A21F01F01002241F068
:10B784000C0140F20110FDF7A1FE0022FF2140F25E
:10B794000110FDF79BFE0022114640F20110FDF757
:10B7A40095FE01220446FF2140F20110FDF78EFEB2
:10B7B40062B644EA002080B210BD70B5044672B689
:10B7C4000022C0F3471140F20110FDF77FFEE100B3
:10B7D40041F00601002201F0FE0140F20110FDF7E4
:10B7E40075FE210A21F01F01002241F00C0140F2F4
:10B7F4000110FDF76BFE0022FF2140F20110FDF75E
:10B8040065FE0022114640F20110FDF75FFE0022A2
:10B814001146064640F20110FDF758FE002211467B
:10B82400054640F20110FDF751FE01220446FF21B6
:10B8340040F20110FDF74AFE62B6240444EA0060B7
:10B84400304340EA052070BD1E4B37B522221A80D2
:10B854001D4B4FF480721A801C4A4FF4805313809E
:10B864001B4A13801B4B1C4A1A601C4B00241C608F
:10B874001B4B02AD1C601B4B05F8014D1C601A4BA1
:10B884002846012240F60F011C70FFF75AFA9DF872
:10B894000730012223F0020340F60F0128468DF8F9
:10B8A4000730FFF7BEFA114B1C70114B1C70114B83
:10B8B4001C70114B1C70114B1C70114B1C7003B08D
:10B8C40030BD00BFC6140020B4140020AC14002006
:10B8D400BE140020C0140020A8120020CC140020A4
:10B8E400B8140020B0140020C8140020AA140020AA
:10B8F400A9140020BC140020C5140020C414002086
:10B90400A814002038B50020FFF788FB104C4388AA
:10B91400104D238003882B800120FFF77FFB0E4A04
:10B9240043880E49138002880A80288821880144AC
:10B93400914202DD1344984207DB0020FFF756FBD7
:10B944000120FFF753FB002038BD162038BD00BF8F
:10B95400C6140020AC140020B4140020BE1400202F
:10B9640037B51A4B002420461C70FFF728FB012032
:10B97400FFF725FB164B174A1A60174B1C60174B31
:10B9840002AD1C60164B05F8014D1C60154B284692
:10B99400012240F60F011C70FFF7D3F99DF8073020
:10B9A400012223F0020340F60F0128468DF80730E8
:10B9B400FFF737FA0C4B1C700C4B1C700C4B1C70B3
:10B9C4000C4B1C700C4B1C7003B030BDAA1400202F
:10B9D400C0140020A8120020CC140020B8140020A9
:10B9E400B0140020C8140020A9140020BC140020A6
:10B9F400C5140020C4140020A8140020084B1B7890
:10BA0400012B437903D103F00F02042A05D103F07B
:10BA14000F03042B01D1FEF7B1B80220704700BF19
:10BA2400740D00202DE9F341254B1B7803F00F031F
:10BA3400012B80463FD0234B1B78002B3BD0224E5A
:10BA44003478002C39D10788204D0637BAB22988BA
:10BA5400FFF7E7F902A8012200F8014D40F60D01B5
:10BA6400FFF76FF99DF807301B070AD4184B298894
:10BA74001B88184819440139012289B20470FFF760
:10BA8400D0F9154D2868804505D080B13A46414625
:10BA940003F058FE2868114B1A6852B1002218604E
:10BAA40001232A603370204602B0BDE8F08140468D
:10BAB400F1E70B4AF3E7F024F5E70724F3E700BFC7
:10BAC4005D0D0020AA140020A9140020BE1400203B
:10BAD400B4140020670D0020C0140020B814002006
:10BAE400A8130020124B002210B51A70114B124CEF
:10BAF4001A681AB1216809B910490A60104A206805
:10BB040012681A6020B1FFF78DFF0023236010BD77
:10BB14000C4A137853B1590608D523F04003137027
:10BB2400064BBDE810401868FEF740B910BD00BFD1
:10BB3400A9140020CC140020B0140020C01400204C
:10BB4400B8140020C5140020F8B50E4B1C6894B13D
:10BB54000D4D2B7863B10D4F3E684EB90120FFF7B0
:10BB64002EFA0B4B01201B683B60FFF73FFA2E7047
:10BB74002046FFF757FF074A1378B3FA83F35B09AC
:10BB84001370F8BDCC140020A9140020B0140020B8
:10BB9400B8140020C814002038B5154B1B7803F0E6
:10BBA4000F03012B0C4621D0124D43792A785207FA
:10BBB40004BF01222A702A7803F00F03437143EA79
:10BBC40002134371FFF72EFF60B144F0800401209B
:10BBD40064B2002C0BDA084B197804F07F040C4390
:10BBE4001C7038BD2B7801332B70F1E7F02038BD81
:10BBF4005D0D0020A8140020C514002010B5018894
:10BC04004379B1F5807F04464FEA13120DD923F02E
:10BC14000F03437101230422C3800823028003819C
:10BC24000021BDE81040FFF7B7BF0B4B12B11978E4
:10BC3400914210D020461A70FFF7E0FE58B1042359
:10BC440023806379208123F00F0363710123E38050
:10BC540000212046E5E710BDC4140020F7B5204CB0
:10BC6400022221880DF10600FFF76BF8BDF80630BB
:10BC74001C4A063311781C4A9BB2ADF8063011B940
:10BC84001A49097819B10123137003B0F0BD184F94
:10BC940011703A88174D21882868934288BFADF8FF
:10BCA4000620BDF80620FFF74CF802A8002600F88D
:10BCB400036D012240F60501FFF743F89DF80530B6
:10BCC4001B0709D521883B880B48194401390122F7
:10BCD40089B20670FFF735F82868FFF78FFFD4E7BD
:10BCE400AC140020A9140020BC140020C5140020AA
:10BCF400C6140020C0140020670D0020024B1B78DE
:10BD04000BB1FFF7ABBF7047BC1400207047002095
:10BD140070470020704700207047002070470020C3
:10BD2400704700207047042303800B800020704775
:10BD3400014B1B680360704760060020014B0268DA
:10BD44005A60704760060020034B5A6812B10132F2
:10BD54001A6070471A68FAE76006002008B50121E6
:10BD64004FF4807000F04AFE00214FF48070BDE86B
:10BD7400084000F043BE43680A7923F0407323F47B
:10BD8400807343EA02230A6813434360CA680B6959
:10BD940013438A6810B513438468084A2240134346
:10BDA4004A7943EA420383600A7DC36A013A23F471
:10BDB4007003D2B243EA0253C36210BDFDF7FFC061
:10BDC40000230360037143718360C3600361012333
:10BDD4000375704790E80C00064910B513434C688E
:10BDE400054A2240134382681343C26813434B60DD
:10BDF40010BD00BF00230140E030FCFF00230360BE
:10BE040043608360C3607047836819B143F00103E2
:10BE14008360704723F00103FAE7436823F4400387
:10BE240023F4007319434160704741628262704792
:10BE3400436823F01F03194341607047044B5A6859
:10BE440018B142F400025A60704722F40002FAE783
:10BE540000230140044B5A6818B142F480025A602E
:10BE6400704722F48002FAE700230140092970B5E3
:10BE74001BD9A1F10A04C56804EB44040726A640B3
:10BE840025EA060503FA04F42C43C460062A18D8EC
:10BE9400013A436B02EB82021F24944023EA040319
:10BEA40001FA02F21A43426370BD056901EB4106CF
:10BEB4000724B44025EA040503FA06F42C4304617C
:10BEC400E4E70C2A0CD8073A036B02EB82021F2426
:10BED400944023EA040301FA02F21A43026370BD98
:10BEE4000D3AC36A02EB82021F24944023EA04033E
:10BEF40091401943C16270BD836843F080438360FD
:10BF04007047836819B143F480638360704723F4F6
:10BF14008063FAE7836819B143F0020383607047D2
:10BF240023F00203FAE74368013923F4604343EA48
:10BF3400413343607047436819B143F4006343607D
:10BF4400704723F40063FAE7C06C80B27047014B7A
:10BF54001868704708230140836819B143F480735B
:10BF64008360704723F48073FAE7836819B143F45C
:10BF740000738360704723F40073FAE7044B5A6834
:10BF840018B142F400525A60704722F40052FAE7A2
:10BF940000230140092970B51CD9A1F10A04C56820
:10BFA40004EB44040726A64025EA060503FA04F434
:10BFB4002C43C460836B0232C3F30154121BD2B20C
:10BFC40002EB82021F24944023EA040391401943A4
:10BFD400816370BD056901EB41060724B44025EA7D
:10BFE400040503FA06F42C430461E3E7836B013987
:10BFF40023F4401343EA01538363704782B0002360
:10C0040001930190019B19440191019B1A6002B0B4
:10C014007047836823F470231943816070478368F1
:10C0240023F44013194381607047836843F4800309
:10C03400836070478068C0F380507047FFF7FABF91
:10C04400436819B143F480634360704723F4806309
:10C05400FAE7436819B143F480534360704723F40B
:10C064008053FAE782B0002301930190019B2833A7
:10C0740019440191019B186880B202B070470123F2
:10C08400C9B203FA01F1436812B119434160704720
:10C0940023EA0101FAE70368194214BF01200020D2
:10C0A4007047C943016070474268006810EA112074
:10C0B40007D00123C9B203FA01F1114214BF184693
:10C0C400002070476FEA112101607047036823F074
:10C0D400010303600023036043608360C360036162
:10C0E400212343612A4B984203D13D2243F8082C73
:10C0F4007047284B984204D14FF4746243F8202CC3
:10C104007047254B984204D14FF4741243F8382CED
:10C114007047224B984204D14FF0746243F8502C7C
:10C1240070471F4B984203D11E4A43F8642C704752
:10C134001D4B984203D11D4A43F87C2C70471C4B7D
:10C14400984203D11B4A43F8942C70471A4B9842E7
:10C1540004D14FF03D5243F8AC2C17E0174B9842F2
:10C16400C3D0174B9842C7D0164B9842CCD0164B2D
:10C174009842D1D0154B9842D6D0154B9842DAD07C
:10C18400144B9842DED0144B9842E2D0704700BF63
:10C194001060024028600240406002405860024043
:10C1A400706002403D00002088600240400F002083
:10C1B400A060024000003D20B860024010640240CC
:10C1C40028640240406402405864024070640240A3
:10C1D40088640240A0640240B86402400368134AC1
:10C1E40010B51A40CC680B6823434C6923438C690F
:10C1F4002343CC6923430C6A23434C6A23438C6A4C
:10C2040023434C6B23438C6B2343134303604269E6
:10C21400CB6A0C6B22F007022343134343610B697F
:10C2240043604B6883608B68C36010BD3F801CF023
:10C234000023036043608360C360036143618361DF
:10C24400C361036243628362C362036343638363C0
:10C254007047036819B143F001030360704723F08A
:10C264000103FAE7036819B143F40043036070471C
:10C2740023F40043FAE7036819B143F02003036091
:10C28400704723F02003FAE741607047406880B2AA
:10C294007047036822B143F40023036001617047CF
:10C2A40023F40023F9E7036819B143F480230360FE
:10C2B400704723F48023FAE70AB101617047C16033
:10C2C40070470068C0F3C0407047006800F0010088
:10C2D4007047406900F0380070470A4B0A4A10B5AD
:10C2E4000A4CA04294BF184610468B004CBF4368CA
:10C2F400036821F0F02121F08211194214BF0120BA
:10C30400002010BD00600240006402400F6402403F
:10C314000B0612D5436952B143F08003802943616F
:10C3240004D0036801F01E0119430160704723F033
:10C3340080038029436104D170478029F6D0002A04
:10C34400EFD1036801F01E0123EA0101EDE7114B6F
:10C35400114A10B5114CA04288BF1A4621F0F023AF
:10C3640023F0C31393B1006800EAD12000F01E0348
:10C3740088004CBF5068106821F0F02121F0821130
:10C38400084002D0181C18BF012010BD436903F0F7
:10C394008003EDE700640240006002400F64024045
:10C3A40010B5084A084B094CA04294BF18461046E1
:10C3B40011F0005F21F0F02121F0821114BFC1605F
:10C3C400816010BD00640240006002400F640240BE
:10C3D400FFF7E6BF044B00221A605A609A60DA60E5
:10C3E400024A5A61704700BF003C0140FFFF7F00D2
:10C3F40082790168037930B542B3194A1568CC4390
:10C4040025401560556803F1804303F59E332C40A5
:10C4140054601C682143196003689468D9430C4034
:10C424009460D4682140D1604179102906D1916883
:10C4340019439160D1680B43D36030BD01F1804250
:10C4440002F59E3211680B43136030BD03F1804343
:10C4540003F59E331A6822EA0101196030BD00BF5A
:10C46400003C014000230C2203600371427183717C
:10C474007047024A1369184310617047003C014039
:10C48400034B5B69034214BF01200020704700BFC7
:10C49400003C0140014B5861704700BF003C014023
:10C4A400054B1A685B69034004D0024214BF0120A3
:10C4B4000020704718467047003C0140014B58610A
:10C4C400704700BF003C014008B5304B984209D189
:10C4D4000121084600F062FA00210120BDE808406D
:10C4E40000F05CBA2A4B984206D10121022000F0E8
:10C4F40055FA00210220F1E7264B984206D101218A
:10C50400042000F04BFA00210420E7E7224B984274
:10C5140006D10121082000F041FA00210820DDE7BE
:10C524001E4B984206D10121102000F037FA002159
:10C534001020D3E71A4B984206D10121202000F0A5
:10C544002DFA00212020C9E7164B984206D101217B
:10C55400402000F023FA00214020BFE7124B98420C
:10C5640006D10121802000F019FA00218020B5E7CE
:10C574000E4B984208D101214FF4807000F00EFA5E
:10C5840000214FF48070A9E708BD00BF00000240FD
:10C594000004024000080240000C02400010024067
:10C5A4000014024000180240001C02400020024017
:10C5B4002DE9F0430D6800220126032406FA02FC4B
:10C5C4003CEA05033DD15700D0F800E004FA07F334
:10C5D400DB430EEA030EC0F800E091F804E0D0F863
:10C5E40000900EFA07F80EF1FF3E48EA0908BEF182
:10C5F400010FC0F8008017D8D0F808E003EA0E0352
:10C6040083604B79D0F808E0BB4043EA0E038360B3
:10C61400436823EA0C0343608B79D0F804E0934029
:10C624009BB243EA0E034360C36804FA07FE23EA9D
:10C634000E03C360CB79D0F80CE0BB4043EA0E0391
:10C64400C3600132102AB9D1BDE8F0834FF6FF73FD
:10C6540003600023037143718371C371704782B017
:10C664004FF480330193019B0B430193019BC361FE
:10C67400C161019BC361C3690193C369019302B0A2
:10C6840070470369194214BF0120002070470069F4
:10C6940080B270474369194214BF012000207047DB
:10C6A400406980B2704701837047418370470AB183
:10C6B4000183704741837047416170474369594022
:10C6C4004161704701F00703C90800EB810010B510
:10C6D400016A9B000F249C4021EA04010162016A63
:10C6E4009A400A43026210BD0A4B1A68002142F0C4
:10C6F40001021A6099601A6822F0847222F480326E
:10C704001A60054A5A601A6822F480221A60D960B5
:10C71400704700BF0038024010300024024B002252
:10C724001A701870704700BF02380240034A136839
:10C7340023F0F80343EAC000106070470038024059
:10C74400014B1860704700BF00004742064B0022AF
:10C7540001281A701A7002D0042802D07047187089
:10C76400704705221A70704770380240014B1860F8
:10C77400704700BF800E474210B5029C40EA046037
:10C7840008435B08013B40EA821040EA0340014B46
:10C79400586010BD00380240014B1860704700BF5C
:10C7A400600047420907034B41EA8011C3F8841033
:10C7B400704700BF00380240014B1860704700BF4B
:10C7C40068004742014B1860704700BF4C00474265
:10C7D400034A936823F0EC63194301439160704763
:10C7E40000380240034A936823F078431943014315
:10C7F4009160704700380240034A936823F00303B2
:10C8040018439060704700BF00380240024B98689C
:10C8140000F00C00704700BF00380240034A9368E0
:10C8240023F0F00318439060704700BF00380240C3
:10C83400034A936823F4E05318439060704700BFA1
:10C8440000380240034A936823F4604343EAC0007B
:10C8540090607047003802401A4A1B4B916801F0FF
:10C864000C01042910B501D0082917D0154A03601A
:10C8740093681649C3F30313CC5C0368E340436035
:10C884009468C4F382240C5D23FA04F484609268EF
:10C89400C2F342328A5CD340C36010BD546851680D
:10C8A4005268C2F3881201F03F01B3FBF1F3534322
:10C8B400044A5268C2F3014201325200B3FBF2F35C
:10C8C400D4E700BF003802400024F40090000020A8
:10C8D40000F44073B3F5407F084A08D1916820F012
:10C8E400704321F4F81123F440730B439360136FE6
:10C8F400C0F30B0018431067704700BF00380240B4
:10C90400014B1860704700BF3C0E4742014B186052
:10C91400704700BF400E4742014B1860704700BF8C
:10C924005C014742044B1A6B11B110431863704702
:10C9340022EA0000FAE700BF00380240044B5A6BB9
:10C9440011B110435863704722EA0000FAE700BFB0
:10C9540000380240044B9A6B11B11043986370473E
:10C9640022EA0000FAE700BF00380240044B1A6CC8
:10C9740011B110431864704722EA0000FAE700BFBF
:10C9840000380240044B5A6C11B11043586470478C
:10C9940022EA0000FAE700BF00380240044B1A699B
:10C9A40011B110431861704722EA0000FAE700BF92
:10C9B40000380240044B5A6911B110435861704762
:10C9C40022EA0000FAE700BF00380240044B9A69EB
:10C9D40011B110439861704722EA0000FAE700BFE2
:10C9E40000380240044B1A6A11B1104318627047B0
:10C9F40022EA0000FAE700BF00380240044B5A6AFA
:10CA040011B110435862704722EA0000FAE700BFF0
:10CA140000380240044B1A6D11B110431865704779
:10CA240022EA0000FAE700BF00380240044B5A6DC6
:10CA340011B110435865704722EA0000FAE700BFBD
:10CA440000380240044B9A6D11B110439865704749
:10CA540022EA0000FAE700BF00380240044B1A6ED5
:10CA640011B110431866704722EA0000FAE700BFCC
:10CA740000380240044B5A6E11B110435866704797
:10CA840022EA0000FAE700BF00380240044B1A789B
:10CA940011B110431870704722EA0000FAE700BF92
:10CAA4000D3802404209012A074B07D11B6800F0E8
:10CAB4001F0023FA00F000F001007047022A0CBFA7
:10CAC4001B6F5B6FF3E700BF0038024007B500231C
:10CAD40001933120FFF7E6FF019B01330193019B92
:10CAE400B3F5A06F01D00028F3D03120FFF7DAFFAF
:10CAF400003018BF012003B05DF804FB024A536FF5
:10CB040043F080735367704700380240034BDB687F
:10CB1400184214BF01200020704700BF00380240B3
:10CB2400014B1870704700BF0E38024008B5154B12
:10CB340098420BD101214FF48050FFF75FFF002191
:10CB44004FF48050BDE80840FFF758BF0E4B9842A1
:10CB54000BD101214FF48040FFF744FF00214FF433
:10CB64008040BDE80840FFF73DBF084B984208D11C
:10CB740001214FF40040FFF735FF00214FF400403E
:10CB8400EFE708BD0030014000380040003C0040A1
:10CB9400038810B503F441524C880B8823438C88D6
:10CBA4002343CC8823430C8923434C8923438C8916
:10CBB4002343CC89234313439BB20380838B23F405
:10CBC40000631B041B0C83830B8A038210BD838BBD
:10CBD40023F47B6323F00F031B041B0C83830223C6
:10CBE40003848B68F0B5848B022BA4B24ED0284EFC
:10CBF4008A88002AB26814BF02270127120242BFA2
:10CC0400B26822F40002B260D6F88420D6F88450C8
:10CC1400D6F804E0C2F388160EF03F0E1D4AB2FBAC
:10CC2400FEF2C5F302757243B2FBF5F5CA88B2F59C
:10CC3400007F08BF2D0A4FF00A021CBF7E01B5FB1E
:10CC4400F6F56A43B2FBF3F305330A229BB2B3FB56
:10CC5400F2F303F001021202C3F34F039D1EADB2BF
:10CC6400FE2D24BF002202231343CA8813439BB220
:10CC74004A8803840B8813438A8843F4006313436C
:10CC84008A8913431C43A4B28483F0BD0022E5E7E0
:10CC9400003802400024F400002303804380838092
:10CCA400C380038143818381C38107230382704747
:10CCB40000230222038043808380C38082608381B7
:10CCC4007047038821B19BB243F04003038070474F
:10CCD40023F040031B041B0CF8E7838B21B19BB2A8
:10CCE40043F480638383704723F480631B041B0C29
:10CCF400F8E7038823F400631B041B0C03800388F8
:10CD04009BB21943018070470388B1F5804F15BF6A
:10CD140023F480439BB21B0443F4804318BF1B0CD1
:10CD2400038070474FF6FF63994203880BBF23F4D7
:10CD340080739BB21B0443F4807308BF1B0C0380F5
:10CD44007047838821B19BB243F00403838070470A
:10CD540023F004031B041B0CF8E7838821B19BB266
:10CD640043F010038380704723F010031B041B0C53
:10CD7400F8E7808980B2704781817047038821B1C8
:10CD84009BB243F400530380704723F400531B0405
:10CD94001B0CF8E703889BB243F48053038070476D
:10CDA400012914BF008B808A80B27047008A80B248
:10CDB400704783889BB212B119438180704723EA7C
:10CDC4000101FAE70B0901219940838889B29BB2DA
:10CDD40012B119438180704723EA0101FAE70389FC
:10CDE400194214BF012000207047C94389B2018150
:10CDF400704710B58488008901F00F02012380B2C6
:10CE040003FA02F21040A4B205D009098B401C4277
:10CE140014BF0120002010BD01F00F03012199402F
:10CE2400C94389B20181704730B5048C24F00104F0
:10CE34002404240C0484048B058C24F0F3042404BB
:10CE440042EA0313240C1C4325F00A031B041B0CA5
:10CE540041F00101A4B20B430483038430BD30B517
:10CE6400048C24F010042404240C0484058B048C06
:10CE7400120242EA033324F0A00225F4407512049E
:10CE84002D05120C2D0D42EA01111D4341F0100134
:10CE9400ADB289B20583018430BD08B54D4B9842CB
:10CEA40009D101210846FFF7A9FD00210120BDE8B1
:10CEB4000840FFF7A3BDB0F1804F09D10121084616
:10CEC400FFF790FD00210120BDE80840FFF78ABD6F
:10CED400414B984206D101210220FFF783FD002136
:10CEE4000220F1E73D4B984206D101210420FFF7CF
:10CEF40079FD00210420E7E7394B984206D101214E
:10CF04000820FFF76FFD00210820DDE7354B98422C
:10CF140006D101211020FFF765FD00211020D3E781
:10CF2400314B984206D101212020FFF75BFD0021FF
:10CF34002020C9E72D4B984206D101210220FFF79A
:10CF44005DFD00210220B2E7294B984208D101215E
:10CF54004FF48030FFF752FD00214FF48030A6E7F4
:10CF6400244B984208D101214FF40030FFF746FDCD
:10CF740000214FF400309AE71F4B984208D1012159
:10CF84004FF48020FFF73AFD00214FF480208EE714
:10CF94001A4B984206D101214020FFF723FD0021BE
:10CFA400402091E7164B984206D101218020FFF7DB
:10CFB40019FD0021802087E7124B984208D10121F6
:10CFC4004FF48070FFF70EFD00214FF480707BE773
:10CFD40008BD00BF000001400004004000080040FC
:10CFE400000C004000100040001400400004014008
:10CFF4000040014000440140004801400018004046
:10D00400001C0040002000401C4A038890429BB250
:10D0140012D002F5806290420ED0B0F1804F0BD056
:10D02400A2F58032904207D002F58062904203D08C
:10D0340002F58062904203D14A8823F070031343BF
:10D044000F4A904208D002F5806290421FBF23F439
:10D0540040730A899BB2134303804B68C3620B88F5
:10D064000385064B984203D003F58063984201D1AF
:10D074008B7A038601238382704700BF000001403E
:10D08400001000404FF0FF3343600023038003810E
:10D09400438083727047018582827047038823F03E
:10D0A40070031B041B0C19430180704741627047D5
:10D0B400C1627047406A7047008D80B27047038830
:10D0C40021B19BB243F002030380704723F00203B3
:10D0D4001B041B0CF8E7038821B19BB243F0040343
:10D0E4000380704723F004031B041B0CF8E7038838
:10D0F40021B19BB243F080030380704723F0800387
:10D104001B041B0CF8E7038823F008031B041B0C07
:10D11400038003889BB2194301807047038823F47A
:10D1240040731B041B0C038003889BB219430180CA
:10D134007047038821B19BB243F001030380704719
:10D1440023F001031B041B0CF8E7038C23F00103F9
:10D154001B041B0C038470B5038C8288048B0D881C
:10D164004E8824F073042404240C2C4323F002037B
:10D174008D891B0435431B0C2B430F4DA84292B2DF
:10D184009BB203D005F58065A8420ED1CD894E8AA5
:10D1940023F008032B438D8823F004032B430D8ACB
:10D1A40022F4407235432A4392B282808A6804830F
:10D1B4004263038470BD00BF00000140038C23F070
:10D1C40010031B041B0C038470B5038C8488028B2E
:10D1D4000D884E8822F4E6421204120C42EA05221B
:10D1E40023F020038D891B0435431B0C43EA0513EC
:10D1F400114DA842A4B292B29BB203D005F580654A
:10D20400A84213D1CD894E8A23F0800343EA051343
:10D214004FF6BF751D408B8845EA03130D8A24F42D
:10D224004064354344EA85049BB2A4B284800283FB
:10D234008A688263038470BD00000140038C23F478
:10D2440080731B041B0C038470B5038C8288848B4D
:10D254000D884E8824F073042404240C2C4323F4F6
:10D2640000738D891B0435431B0C43EA0523114DC0
:10D27400A84292B29BB203D005F58065A84213D1AF
:10D28400CD894E8A23F4006343EA05234FF6FF3524
:10D294001D408B8845EA03230D8A22F4405235430E
:10D2A40042EA05129BB292B282808A688483C26386
:10D2B400038470BD00000140038C23F480531B04DD
:10D2C4001B0C038470B5038C8488828B0D884E8874
:10D2D40022F4E6421204120C42EA052223F400531B
:10D2E4008D891B0435431B0C43EA05330A4DA842C0
:10D2F400A4B292B29BB203D005F58065A84205D1D1
:10D304000D8A24F4804444EA8514A4B28480828380
:10D314008A680264038470BD000001400023038016
:10D324004380838083608381C38103824382704707
:10D3340030B5048C0125A4B28D4024EA050400F123
:10D344001803048421F0080050B94908C85820F093
:10D3540070000004000CC850C8580243CA5030BDC5
:10D364000439C1F34E011202C85820F4E04000040D
:10D37400000CC85092B2C858EFE74163704781630C
:10D384007047C163704701647047038B23F07003D7
:10D394001B041B0C194301837047038B23F4E043E4
:10D3A4001B041B0C43EA012189B201837047838B60
:10D3B40023F070031B041B0C194381837047838B78
:10D3C40023F4E0431B041B0C43EA012189B281834B
:10D3D4007047038B23F008031B041B0C19430183C0
:10D3E4007047038B23F400631B041B0C43EA0121E5
:10D3F40089B201837047838B23F008031B041B0C41
:10D40400194381837047838B23F400631B041B0C33
:10D4140043EA012189B281837047038B23F004031B
:10D424001B041B0C194301837047038B23F4806393
:10D434001B041B0C43EA012189B201837047838BCF
:10D4440023F004031B041B0C194381837047838B53
:10D4540023F480631B041B0C43EA012189B28183FA
:10D464007047038B23F080031B041B0C19430183B7
:10D474007047038BC3F30E0343EA012189B201838E
:10D484007047838B23F080031B041B0C1943818397
:10D494007047838BC3F30E0343EA012189B281836E
:10D4A4007047038C23F002031B041B0C19430184F3
:10D4B4007047038C23F008031B041B0C19430184DD
:10D4C4007047038C23F020031B041B0C43EA011157
:10D4D40089B201847047038C23F080031B041B0C66
:10D4E40043EA011189B201847047038C23F4007369
:10D4F4001B041B0C43EA012189B201847047038C8D
:10D5040023F400631B041B0C43EA012189B2018448
:10D514007047038C23F400531B041B0C43EA0131B2
:10D5240089B201847047038C10B501248C409BB2EE
:10D5340023EA04030384038C02FA01F1194389B238
:10D54400018410BD038C10B504248C409BB223EAE3
:10D5540004030384038C02FA01F1194389B20184A0
:10D5640010BD00230122038043808280C380038195
:10D574007047406B7047806B7047C06B7047006C9E
:10D584007047038B23F00C031B041B0C0383038BD6
:10D594009BB2194301837047038B23F440631B043C
:10D5A4001B0C0383038B9BB243EA012189B20183E1
:10D5B4007047F8B50C464988A288B4F800E023897E
:10D5C40000290CBF02260026012A0CBF02270127CE
:10D5D400BEF1000F0ED1FFF727FCE188FFF7D1FF62
:10D5E400314623893A46FFF73AFCE188BDE8F84022
:10D5F400FFF7D2BFFFF733FCE188FFF7CDFF3146D9
:10D6040023893A46FFF710FCE188BDE8F840FFF7AC
:10D61400B8BF838B23F00C031B041B0C8383838B05
:10D624009BB2194381837047838B23F440631B04AB
:10D634001B0C8383838B9BB243EA012189B28183D0
:10D644007047F8B50E880B898A880D46498836B923
:10D65400FFF7EAFBE988BDE8F840FFF792BF042E24
:10D6640006D1FFF7FCFBE988BDE8F840FFF794BF5B
:10D67400082EEF88058C1CD125F480752D042D0C03
:10D684000584868B058CB6B226F0F3063243ADB220
:10D6940042EA031325F4206242F4807242EA012232
:10D6A4009BB292B2838339460284BDE8F840FFF707
:10D6B400B0BF25F480552D042D0C0584868B058C74
:10D6C4001B0343EA022326F4407645F6FF722A4000
:10D6D4003605360D42F48052334342EA01329BB29E
:10D6E40092B2838339460284BDE8F840FFF79CBFB9
:10D6F4004A880B8813438A881343CA8813430A89C8
:10D7040013434A8913438A8913439BB2A0F84430D4
:10D7140070470023038043808380C3800381438157
:10D7240083817047B0F8443039B16FEA43436FEAFC
:10D7340053439BB2A0F844307047C3F30E03F9E798
:10D74400838821B19BB243F004038380704723F0A4
:10D7540004031B041B0CF8E7838821B19BB243F03C
:10D7640001038380704723F001031B041B0CF8E7BB
:10D7740081827047038A194214BF01200020704738
:10D78400C94389B201827047038A828911EA03007E
:10D7940092B203D0114214BF012000207047C94344
:10D7A40089B2018270470A43A0F8482070478389F0
:10D7B4009BB212B119438181704723EA0101FAE750
:10D7C400FFF7F5BF838821B19BB243F00803838040
:10D7D400704723F008031B041B0CF8E7038923F0AC
:10D7E40007031B041B0C03817047038923F0700398
:10D7F4001B041B0C1943018103899BB243F00703EB
:10D804000381704738B50D46602D114604464FF02C
:10D8140001020ED1FFF723FB218921F070010904D5
:10D82400090C2943218123899BB243F007032381F7
:10D8340038BDFFF7F9FAEFE7038923F070031B04FF
:10D844001B0C194301817047838823F070031B0468
:10D854001B0C838083889BB21943818070470389A2
:10D8640023F007031B041B0C038103899BB2194398
:10D8740001817047038923F080031B041B0C03817F
:10D8840003899BB219430181704710B504890A4387
:10D89400E4B242EA03231C43A4B2048110BD10B5D0
:10D8A400FFF7F3FF038923F077031B041B0C43F0FA
:10D8B4007703038110BD10B5FFF7E7FF03899BB21F
:10D8C40043F48043038110BD70B50689048B058C35
:10D8D40024F4407424F0030425F0220526F00706FE
:10D8E40024042D043604240C2D0C42EA0313360CB4
:10D8F40044F480741D43314344F00104ADB201810A
:10D904000483058470BD838821B19BB243F08003F6
:10D914008380704723F080031B041B0CF8E7A0F8F6
:10D924005010704708B5254B984209D101211020A9
:10D93400FFF764F800211020BDE80840FFF75EB847
:10D944001F4B98420BD101214FF40030FFF74AF8E6
:10D9540000214FF40030BDE80840FFF743B8194BED
:10D96400984208D101214FF48020FFF73BF80021B1
:10D974004FF48020EFE7144B984208D101214FF473
:10D984000020FFF72FF800214FF40020E3E70F4BAE
:10D99400984208D101214FF48010FFF723F80021A9
:10D9A4004FF48010D7E70A4B984206D1012120207A
:10D9B400FFF724F800212020BEE708BD0010014035
:10D9C4000044004000480040004C0040005000402B
:10D9D40000140140028A30B50D4692B2EB88898961
:10D9E40022F440521A4302828389044623F4B0523B
:10D9F4002889AB880343688922F00C02034312048C
:10DA0400120C9BB21343A381A38A9BB223F44073E9
:10DA14000B4385B0A3826846FEF71EFF194B9C4258
:10DA240003D003F580639C4222D10399A38913F4A4
:10DA3400004F2B684FF0190214BF5B009B004A4350
:10DA4400B2FBF3F1A28964251204B1FBF5F34FEAAA
:10DA5400031005FB13130DD5DA003232B2FBF5F2D5
:10DA640002F0070242EA00039BB2238105B030BDF5
:10DA74000299DBE71B013233B3FBF5F303F00F0329
:10DA84000343F1E7001001404FF4165303600C22E6
:10DA940000238380C3800381428183817047038A8A
:10DAA4009BB223F4706210B50B884C8823438C8896
:10DAB400C98823430B439BB21343038210BD002345
:10DAC400038043808380C3807047838921B19BB2E4
:10DAD40043F400538381704723F400531B041B0C4D
:10DAE400F8E7038B03F47F430383038B9BB219434F
:10DAF40001837047838931B16FEA43436FEA53432B
:10DB04009BB283817047C3F30E03FAE7838A21B182
:10DB14009BB243F400638382704723F400631B04C5
:10DB24001B0CF8E7C1F30801818070478088C0F3BB
:10DB340008007047038A23F00F031B041B0C0382A5
:10DB4400038A9BB2194301827047838921B19BB236
:10DB540043F002038381704723F002031B041B0C70
:10DB6400F8E7838923F400631B041B0C83818389F6
:10DB74009BB2194381817047038A23F020031B045D
:10DB84001B0C0382038A9BB2194301827047038AE8
:10DB940021B19BB243F480430382704723F4804352
:10DBA4001B041B0CF8E783899BB243F001038381B8
:10DBB4007047838A21B19BB243F008038382704784
:10DBC40023F008031B041B0CF8E7038BDBB203836D
:10DBD400038B9BB243EA012101837047838A21B1FD
:10DBE4009BB243F020038382704723F020031B047D
:10DBF4001B0CF8E7838A21B19BB243F010038382A4
:10DC0400704723F010031B041B0CF8E7838A23F0EE
:10DC140004031B041B0C8382838A9BB219438182F5
:10DC24007047838A21B19BB243F002038382704719
:10DC340023F002031B041B0CF8E7838A9BB212B186
:10DC440019438182704723EA0101FAE710B5C1F351
:10DC5400421401F01F03012C4FF0010101FA03F1FA
:10DC640005D10C3003683AB11943016010BD022C90
:10DC74000CBF10301430F5E723EA0101F5E70388FF
:10DC8400194214BF012000207047C94389B20180A2
:10DC94007047C1F3421210B5012301F01F04012A99
:10DCA40003FA04F30ED1828992B21340028892B22D
:10DCB4006BB10123090A03FA01F10A4214BF1846A1
:10DCC400002010BD022A0CBF028A828AECE71846A3
:10DCD40010BD0B0A01219940C94389B201807047E4
:10DCE40040F0BF60024B40F40030D860704700BF82
:10DCF40000ED00E010B5C3780278FBB1154BD9688C
:10DD040043788078C943C1F30221C1F10404E4B229
:10DD1400A3400F2444FA01F10140DBB20B430E4946
:10DD24001B018818DBB280F800335009012302F08C
:10DD34001F0203FA02F241F8202010BD5309012109
:10DD440002F01F0201FA02F22033034941F82320B2
:10DD540010BD00BF00ED00E000E100E021F06041F3
:10DD640021F07F01014B01439960704700ED00E011
:10DD7400044B1A6911B110431861704722EA00007C
:10DD8400FAE700BF00ED00E0044B1A6804280CBF5A
:10DD940042F0040222F004021A60704710E000E02E
:10DDA40010B5D0F8E83504461B699847032384F876
:10DDB4001231002010BD08B590F8123180F81331EB
:10DDC400042380F81231D0F8E835DB689847002046
:10DDD40008BD08B5D0F8E435DB6903B198470020E5
:10DDE40008BD08B5D0F8E4351B6A9847002008BD83
:10DDF40008B5D0F8E4355B6A9847002008BD10B533
:10DE0400D0F8E83504465B699847012384F8153156
:10DE1400002010BDD0F8E83510B504469B6998473A
:10DE2400D4F8E43500215B6820469847002084F844
:10DE3400150110BD002310B519460446402201F017
:10DE440031F9402280210023204601F02BF90123DF
:10DE540084F81231D4F8E835A0785B68984700203C
:10DE640010BD13B56946044600F014FC9DF800107B
:10DE740001F01F03012B0FD007D3022B11D001F0A7
:10DE84008001204601F08EF903E06946204600F047
:10DE94006FFA002002B010BD6946204600F084FBF2
:10DEA400F7E76946204600F097FBF2E738B50446E9
:10DEB400002949D190F81131022B17D1D0F838211B
:10DEC400D0F824319A421ED9C178012908BFD0F86C
:10DED4002811A2EB030204BF5B18C0F82831C0F874
:10DEE4003821D0F8281192B200F0F0F994F81631E4
:10DEF400012B06D11A4A236912685A60002384F858
:10DF04001631002038BDD0F83C21B2FBF3F503FBF9
:10DF140015255DB9934209D8D0F840319A4205D20B
:10DF24002A4600F0D3F9C4F84051DFE7D4F8E435C9
:10DF3400DB682BB194F81221032A01D120469847BB
:10DF4400204600F0F2F9D1E7D0F8E4355B69002B04
:10DF5400D7D090F81221032AD3D19847D1E700BF34
:10DF6400D014002010B5044669BB90F81131032B7E
:10DF74001AD1D0F89033D0F87C23934216D9C178C3
:10DF8400012908BFD0F88013A3EB020304BF89184A
:10DF9400C0F880139A4228BF1A46C0F8903392B250
:10DFA400D0F8801300F0AAF9002010BDD0F8E435B1
:10DFB4001B6923B190F81221032A00D19847204607
:10DFC40000F0A4F9F0E7D0F8E4359B69002BEBD01E
:10DFD40090F81221032AE7D19847E5E72DE9F041AB
:10DFE4000446164698460D46069FFBF7ACF82046B5
:10DFF4002946C4F8E485C4F8E875C4F8EC6501F072
:10E0040003F8D4F8E8351B6898472046BDE8F0418A
:10E01400FBF7ECB800207047D0F8E43510B504469F
:10E024001B689847D4F8E8359B689847002010BDD2
:10E0340008B5D0F8E4355B689847002008BD00BFF8
:10E0440010B5074C2068FF2807D0064B064A9B688A
:10E05400126806499847FF232360002010BD00BFC3
:10E06400D00000206800002068060020571500201A
:10E0740043230B8000487047D400002038B51B4B65
:10E084005A68052A02F10104194602D05C60002096
:10E0940038BD0A7A0023012A4B60F8D0CA68B2F569
:10E0A400006F08BFCB60CC680B699C4202D100238F
:10E0B4000B72ECE78CBFC4F500631B1B4B614D690D
:10E0C400402DA2B20CD94034403DCC604D61402378
:10E0D40001240C7206490A44812101F043F8D6E771
:10E0E4002C44CC600024ABB24C61F1E768060020FC
:10E0F4005F15002038B5282303FB0101074D084BA9
:10E10400B1F88C131B6904462846984740232A46D5
:10E114000121204601F000F8002038BD1715002029
:10E1240068000020F8B50A7812F0600406460D462F
:10E1340028D0202C22D1CC884B78C4B112060BD520
:10E14400214A2249976818462246B847EA881F4957
:10E15400304600F0ABF807E01D4A1C4913601D4B24
:10E1640022461C6000F0BAF800242046F8BD164A86
:10E174002146956818462246A847F6E700F0ACFA0F
:10E184000224F2E74B780A2B10D00B2B13D0062B6A
:10E19400EBD14B881B0A212B05D1CA880E493A2A98
:10E1A40028BF3A22D4E70D493A22D1E701220C498B
:10E1B40000F07CF8D9E78B7813B9064A9361D3E76A
:10E1C40000F08AFAD1E700BF68000020571500204C
:10E1D400D000002068060020E6000020DD000020BA
:10E1E4008006002010B58121044600F07EFF012145
:10E1F400204600F07AFF8221204600F076FF024B91
:10E204005B689847002010BD6800002038B54022A4
:10E2140004460223812100F045FF0223402201210C
:10E22400204600F03FFF822103230822204600F00D
:10E2340039FF084B022200251A715D71064B1B68D9
:10E2440098474023054A0121204600F065FF2846EF
:10E2540038BD00BF0400002068000020171500200E
:10E2640038B5104C237A012B02D1616911B921729E
:10E27400002038BD40290CD9E36840399AB24033B4
:10E28400E3606161402308490A44812100F06AFF88
:10E29400EEE7E5688BB22944E1600021AAB261612E
:10E2A400F1E700BF680600205F15002010B50446A2
:10E2B4001346C4F83C21C4F83821022280F8112105
:10E2C4000A46002100F04EFF002010BD08B5134699
:10E2D4000A46002100F046FF002008BD10B50446A0
:10E2E4001346C4F89423C4F89023032280F8112120
:10E2F4000A46002100F010FF002010BD08B51346A7
:10E304000A46002100F008FF002008BD10B50423D0
:10E3140080F81131002304461A46194600F022FF02
:10E32400204600F09DFD002010BD10B5052380F8A7
:10E334001131002304461A46194600F0EDFE20462A
:10E3440000F08EFD002010BD282303FB0101B1F86D
:10E354008C03704710B58021044600F023FF20464B
:10E36400002100F01FFF2046BDE8104000F078BDFA
:10E3740037B54B7804460D46092B73D8DFE813F004
:10E38400C20000017200D200720067000A0072002D
:10E39400B40087004B881A0A013A062A62D8DFE8DB
:10E3A40002F00426326161616100D0F8EC358078B6
:10E3B4001B680DF106019847EB88402B03D094F8B5
:10E3C4001231012B02D10823ADF80630BDF8062026
:10E3D400002A57D0EB88002B54D09A4228BF1A4603
:10E3E400ADF8062001462046FFF760FF4AE0D0F86A
:10E3F400E43580789B6A0DF1060198470223437047
:10E40400C4F8F005E2E7DBB2052B2BD8DFE803F014
:10E41400030B0F13171BD0F8EC355B68A0780DF1D4
:10E4240006019847D2E7D0F8EC359B68F6E7D0F8B8
:10E43400EC35DB68F2E7D0F8EC351B69EEE7D0F891
:10E44400EC355B69EAE7D0F8EC359B69E6E78B8845
:10E4540043B9CB8833B990F812318D78032B05F08A
:10E464007F0503D12046FFF775FF0BE080F81451B8
:10E47400294600F0D5FE2046FFF748FF2DB10223C0
:10E4840084F81231002003B030BD0123F8E7897805
:10E49400414D01292970E5D890F81231022B0DD095
:10E4A400032BDFD1B1B9022380F8123180F81011A7
:10E4B400FFF7BEFD2046FFF729FFE3E70029F9D067
:10E4C4000121032380F8101180F812312046FFF750
:10E4D400A3FDEFE790F810110129EBD0FFF7A8FD99
:10E4E400297884F81011F1E7CA88012ABAD190F882
:10E4F4001231022B04D0032BB4D100F5887172E7DA
:10E50400264970E790F81231023B012BAAD8224B1E
:10E5140001229A60D0F818210AB103229A600222DB
:10E524001F4960E74B88012B08D1C4F81831D4F88F
:10E53400E43529469B6820469847BBE7022BA1D1C6
:10E544008B8813F0FF0F9DD102691B0A013B5268AF
:10E55400042B07D8DFE803F0030C0E10120001238C
:10E5640063F306120F4B1A60012384F81631A1E7F6
:10E574000223F5E70323F3E70423F1E70523EFE799
:10E5840090F81231023B012B3FF66CAF4B88012B04
:10E594007FF478AF0023C8E78406002088060020B3
:10E5A4008C060020D014002038B590F81231032BCB
:10E5B40004460D460DD10B79012B0AD8D0F8E43569
:10E5C4009B689847EB8813B92046FFF79FFE00200D
:10E5D40038BDFFF7BFFEFAE738B50D468B886A7879
:10E5E400012A0446D9B21CD029D3032A17D190F8A2
:10E5F4001231022B3ED0032B02D0FFF7ABFE0EE00C
:10E604006B881BB94B0601D000F0CCFDD4F8E4357F
:10E6140029469B68204698472046FFF777FE00204E
:10E6240038BD90F81231022B24D0032BE5D16B882E
:10E63400002BF4D14A06EFD000F0CDFDE6E790F8C8
:10E644001221022A16D0032AD7D113F0800F4FF0DB
:10E6540028020E4B15D001F07F0102FB010191F855
:10E664001E2162B10122DA60094902222046FFF725
:10E674001DFED4E74B06D2D000F094FDCFE7002274
:10E68400F1E702FB010191F87623EAE78406002012
:10E694009006002090F8CC350B7090F8CD354B7077
:10E6A40090F8CF2590F8CE3503EB02234B8090F8F9
:10E6B400D12590F8D03503EB02238B8090F8D32535
:10E6C40090F8D23503EB02239BB2CB80C0F84031E3
:10E6D400012380F81131704710B58021044600F001
:10E6E40061FD2046002100F05DFD2046BDE810409C
:10E6F40000F0B6BB30B588B105462B1A15F8014BAE
:10E70400DBB2002CF9D15B00023313800B700323BE
:10E714004B700138022310F8015F05B930BD5A1C53
:10E72400D2B2CD540233DBB28C54F4E737B50023B4
:10E73400104C019305460320FAF76EFD2B68013C4B
:10E744001A69019213D0019A002AF4DA019A42F06C
:10E7540001020192019A1A61064A19690191013A6A
:10E7640002D00199C907F8D40320FAF755FD002017
:10E7740003B030BD410D030010B5C47844B900EBBB
:10E7840082000333D0F8D0009B102246934201D17B
:10E79400002010BD51F8224004600132F6E710B5A4
:10E7A4000332D0F8D03092100020904202D101EB15
:10E7B400800010BD1C6841F820400130F5E70122BB
:10E7C40030B50023827001294FF04002C37082806B
:10E7D4003CD108230370042343704FF4A073C38017
:10E7E40002230372C1724FF0A04303F50062026179
:10E7F4004278C36003EB421203F5106100F1180480
:10E8040002F5106291422DD103F580624261044603
:10E8140003F58862C0F8CC2014F8902B03EB421562
:10E8240003F5A06105F5A065A94222D103EB0232EC
:10E8340003F5805100F1D00402F5805291421CD1BD
:10E8440003F56063C0F80C31002030BD0029CCD141
:10E854000C230370062343704FF4A063C380C1727A
:10E86400084BC2E744F8041B01F50075A563203189
:10E87400C8E744F8041B2031D6E744F8041B01F52B
:10E884008051DBE70000044038B5037A012B0546CC
:10E894004FF0000450F80C2F2AD1936B697A64F37B
:10E8A400104309B143F480139363D3686FF3861361
:10E8B4006FF396536FF351436FF3D343D360FFF772
:10E8C40035FFEB78012B06D1052363F34404EB6891
:10E8D40044F020049C60EB78012B07D1EB689C6822
:10E8E400052262F3440444F020049C60002038BDF7
:10E8F400D36843F04003D360FFF718FF6B7AEA68EC
:10E90400002B0CBF4FF450234FF4E81393631420EF
:10E91400FAF78CFCDFE7C268936843F00103936065
:10E9240000207047C268936823F0010393600020BD
:10E93400704707B500230193019B43F02003019323
:10E94400019B61F38A130193C268019B1361074B16
:10E9540011690191013B02D001998906F8D4032081
:10E96400FAF75AFC002003B05DF804FB410D0300E4
:10E9740007B500230193019B43F010030193C26880
:10E98400019B1361074B11690191013B02D001996D
:10E99400C906F8D40320FAF73FFC002003B05DF861
:10E9A40004FB00BF410D0300C26808B5D368012908
:10E9B4006FF35D736FF39E7307D143F00053D3601D
:10E9C4003220FAF733FC002008BD0029F7D143F0C8
:10E9D4008043F4E7C368586900F001007047C368D6
:10E9E4005869C04300F001007047C368586900F0DB
:10E9F40001007047C36858699B6918407047C36831
:10EA0400586870470269136861F301031360704723
:10EA140010B5C26800236FF080414FF0FF3493615A
:10EA240051615460516109499161C178994208BFAB
:10EA3400102343F0804343F47013916943F460530B
:10EA440043F00C030B439361002010BD00080080C9
:10EA5400F8B5D0F80C31026900261E60136866F31D
:10EA6400CC231360C37A012B04463546374622D1A2
:10EA74000321FFF7C7FF2021C368A020802261F390
:10EA84001F4660F30F055A6262F31F4562F30F06D7
:10EA94004FF490729E62C3F8045162F30F0561F360
:10EAA4001F454FF4A072C3F8085162F30F0567F3D2
:10EAB4001F45C3F80C5110212046FFF73AFF2046AA
:10EAC400FFF756FF226900234FF0FF3113615361B2
:10EAD4009161D3616678216904F118051F464FF0EE
:10EAE400FF0EB34218D3002304F154051E46FF273A
:10EAF400627893421ED30B6943F480730B61E3780D
:10EB0400012B01BF124B402262F359430B63204691
:10EB1400FFF77EFF0020F8BD55F8042B106800288D
:10EB2400ACBF00204FF09040106001331761C2F871
:10EB340008E0D6E755F8042B10680028ACBF002085
:10EB44004FF090401060013316619760D0E700BF2A
:10EB54000301010003699B68C3F34103022B04D042
:10EB640001D8012B03D102207047012070470320F4
:10EB740070470369806999680268C1F341010229F9
:10EB84000ABF03216FF30A0261F30A0202605A68A2
:10EB940042F480725A600020704730B54C780B788C
:10EBA400012C4FF000021DD100EB830504FA03F39E
:10EBB400AD6963F30F022B681C040DD48C6864F3F5
:10EBC4000A03CC78C98864F3934361F3995343F0FF
:10EBD400805343F400432B600369D9690A43DA6123
:10EBE400002030BD00EB8304656D012404FA03F3B7
:10EBF40063F31F42DFE730B54A780B780025012A1A
:10EC04002C4610D100EB830102FA03F3896963F304
:10EC14000F0402696FF3CF350D60D36923EA04034F
:10EC2400D361002030BD00EB8302516D012202FA52
:10EC340003F363F31F44ECE7F8B54F780A784B69A4
:10EC4400012F42D100EB8204A6693468356963F36D
:10EC54001205EBB967F3DC453561C578012D26D182
:10EC64000D697561CD78012D07D10769BF68FF056E
:10EC740054BF44F0005444F0805444F00444012D43
:10EC8400346003D19BB2C968FFF776FD0020F8BD5C
:10EC9400D1F808E003EB0E07013FB7FBFEF767F37B
:10ECA400DC45CF78012F08BF67F35E75D4E7CD78D4
:10ECB400012DD7D0002BD5D007690125D7F834E032
:10ECC400954045EA0E057D63CCE700EB8202566D64
:10ECD4008A6834683569ABB962F31205012363F3BA
:10ECE400DC453561C378012B04BF0B697361CB78B4
:10ECF400012B03D14B798BB144F0005444F004440C
:10ED04003460C3E71344013BB3FBF2F363F3DC4524
:10ED1400C3F30903534363F31205E2E744F0805459
:10ED2400ECE7F7B54F784E69012F3AD185692C6825
:10ED34002B690093DAB2C3F3074316BB66F30602EA
:10ED44008DF8002067F3C4038DF80230009B2B611B
:10ED5400C278012A05D10B780E6900EB83039B6905
:10ED64005E6144F004442C6042B94B6933B10269DA
:10ED74000978506B01238B4003435363002003B095
:10ED8400F0BD8F68BE428CBF67F3060266F30602CD
:10ED94008DF800204FF0010288BF4F6162F3C40375
:10EDA400D2E70B788F6800EB83035D6D2C682B69C9
:10EDB4000093DAB2C3F307439EB967F306028DF8F2
:10EDC4000020012262F3C4038DF80230009B2B6102
:10EDD400C378012B04BF0B696B6144F004442C60BD
:10EDE400CCE74F61E9E74B78012B0B7800EB83000C
:10EDF4000AD182691368002B01DA43F0804343F49B
:10EE04000013136000207047426D1368F7E74B78D6
:10EE1400012B0B78C97800EB8300A1F102010CBF30
:10EE24008269426D136801296FF3555398BF43F00B
:10EE3400805313600020704703699869DB691840A8
:10EE4400000C704700EB81014B6D9A6803695869A7
:10EE54001040704703699869DB69184080B27047B5
:10EE640082B000230093C0238DF8033001224FF0B9
:10EE7400000362F3C4038DF8023018238DF80030C8
:10EE8400436D009A1A61C278012A06D100F2CC506F
:10EE940058611A684FF080221A6002B07047D0F8A7
:10EEA400183110B50446D3B102699368DB0716D54F
:10EEB400837A43B1D0F80C31D0F80C116FF34103CD
:10EEC4006FF300030B60536843F0010353600520A4
:10EED400FAF7ACF92269536823F00103536010BDBB
:10EEE400837A63B103699B68DB0708D5D0F80C31DA
:10EEF400D0F80C216FF341036FF3000313607047E4
:10EF040038B50123044680F81231407804F1180220
:10EF14000023FF21834210D3236900221A615A611E
:10EF2400DA614FF0FF329A612046FFF721FD204657
:10EF34001021BDE83840FFF7FCBC52F8045BA9601F
:10EF4400956B0133A960E5E74B78012B0B7800EB57
:10EF540083000BD183691B68C3F30743990613D459
:10EF640013F0020F14BF202030207047436D1B683C
:10EF7400C3F307439A0609D413F0020F14BF4FF4E6
:10EF840000504FF440507047102070474FF48050A9
:10EF9400704770B44B78012B0B7806460D4600EB96
:10EFA400830316D19C69102A236802D170BCFFF731
:10EFB4001ABF202A02D143F0006311E0302A1DD188
:10EFC4009A0216D500236B712946304670BCFFF7B0
:10EFD4001EBF5C6DB2F5805F236804D143F4001357
:10EFE400236070BC7047B2F5005FE4D0B2F5405FB7
:10EFF400E5E743F0044343F40043F1E7002AEFD18B
:10F0040062F3CF33ECE700BF70B50446FFF7D7FBDC
:10F0140000230121657884F8121184F8143104F571
:10F024008E7218464026AB4202F128021AD30022FF
:10F0340004F55D7311464020AA4203F1280321D34D
:10F044002046FFF76FFC2046FFF71EFC00212046F8
:10F05400FFF7AAFC2046FFF7FBFC2046BDE8704002
:10F06400FFF759BC02F8283C22F8223C02F8271C7E
:10F0740002F8250C42F8206C42F81C0C42F8140CDF
:10F084000133D0E703F8282C23F8222C03F8271C9B
:10F0940003F8251C43F8200C43F81C1C43F8141CEB
:10F0A4000132C9E770B54EB201F07F04002E4FF073
:10F0B4002805B5BF05FB040105FB010101F58E71AF
:10F0C40001F55D71E4B2002EB8BFCC80022BCB7089
:10F0D4004FEAD67508BF00230C704D708A6008BFD4
:10F0E4000B71FFF75AFD002070BD4BB2002B10B519
:10F0F4004FF0280201F07F04B5BF02FB040102FBBC
:10F10400010101F58E7101F55D71DB0F0C704B701F
:10F11400FFF771FD002010BD70B501F07F042826B3
:10F1240006FB040506FB0401C5F88833002385F8B3
:10F134007443C5F88023C5F88C3385F87533C378D8
:10F1440006FB0404012B08BFC5F8842394F8743328
:10F1540001F55D711BB9FFF7E4FD002070BDFFF7F9
:10F164006BFDFAE770B501F07F05282404FB050167
:10F1740004FB05040126C4F82821C4F82C2100222C
:10F1840001F58E7184F81D6184F81C51C4F8342192
:10F19400C4F830311DB9FFF7C4FD002070BDFFF77E
:10F1A4004BFDFAE74BB2002B10B54FF0280201F0EB
:10F1B4007F04B5BF02FB040102FB010101F58E715E
:10F1C40001F55D710122DB0F8A700C704B70FFF743
:10F1D4000AFE002010BD38B54BB2002B01F07F05AC
:10F1E4004FF02802B5BF02FB050102FB010101F546
:10F1F4008E7101F55D710024DB0F8C700D704B7006
:10F20400FFF705FE204638BD08B50B0605D501F00D
:10F214007F01FFF78EFB002008BDFFF7A9FBFAE78B
:10F224000269002361F30A1311680B4313607047EA
:10F23400026953686FF3410353600320F9F7F6BF83
:10F244000269536843F0020353600320F9F7EEBFE9
:10F2540011F0800F4FF028031BBF01F07F0103FB67
:10F26400010103FB010101F58E7108BF01F55D7118
:10F27400FFF76ABE11F0800F4FF028031BBF01F0A7
:10F284007F0103FB010103FB010101F58E7108BF3E
:10F2940001F55D71FFF77DBE2DE9F04F85B00446A1
:10F2A400FFF79DFB18B9002005B0BDE8F08F20469C
:10F2B400FFF7A0FB05460028F5D0C0F3074A1AF073
:10F2C40008000ED02046FFF7B7FDDFF8C0B2814634
:10F2D40004F154074FF00008B9F1000F40F00E811B
:10F2E40001201AF0040F0DD02046FFF7B3FD04F1FE
:10F2F4001807824626464FF00009BAF1000F40F085
:10F3040049810120EEB2B70742BFE36802225A6185
:10F31400002D19DAA37A43B1D4F80C31D4F80C21B6
:10F324006FF341036FF3000313602269536823F002
:10F3340001035360954B1B6820469B699847E3681B
:10F344004FF000425A610120C5F3072739072DD534
:10F3540000238DF80F3094F812318DF80F308B4B59
:10F364001B6820465B6998472369E2689B684FF4F1
:10F3740000615161A27AC2B1DA0716D594F8153149
:10F38400012B12D19DF80F30032B0ED1D4F80C3180
:10F394001A6842F001021A601A6842F003021A6005
:10F3A4007B4A136943F0060313610120330708D530
:10F3B400764B1B682046DB689847E36808225A614D
:10F3C4000120F10615D5E3689A6922F010029A61CA
:10F3D4001E6AC6F34343022B06F00F0900F079813D
:10F3E400062B00F09281E268936943F01003936165
:10F3F4000120FA0631D5226953684FF0000823F042
:10F404000103536041462046FFF793FA667804F1FE
:10F4140018024346FF21B342C0F0848123690126C8
:10F424004FF0FF3266F30F089A6166F31F480B2210
:10F43400C3F81C805A611A611A686FF30A121A60C1
:10F444002046FFF70DFDE3684FF480525A614F4B9D
:10F454001B6820461B6998473046BB0618D52046D2
:10F46400FFF787FBE3682046DE68FFF773FB03289A
:10F4740040F05F810023A3704FF40073A38009233D
:10F4840063F38D26E3684FF40052DE6001205A6175
:10F49400C5F30746F70609D53C4B1B682046DB69D4
:10F4A4009847E3684FF480125A610120B60609D5E3
:10F4B400364B1B6820461B6A9847E3684FF40012DA
:10F4C4005A610120690009D5304B1B6820465B6AEC
:10F4D4009847E3684FF080425A6101206A077FF53C
:10F4E400E3AEE3685D686B0704D5284B1B682046D0
:10F4F4009B6A9847E36801205D60D5E619F0010F27
:10F504003ED05FFA88F3194620460193FFF79AFC30
:10F51400C107064624D53A68019B01269660E17826
:10F52400B1420AD11069282202FB0842C0F312003A
:10F53400D2F87C13091AC2F88C13DBF800201946A0
:10F54400126820469047E378012B09D1B8F1000FE7
:10F5540006D194F81131052B02D12046FFF780FC27
:10F56400B20741BF02263B6832469A60330707D58B
:10F57400DBF8003020469B6898473B6808229A6075
:10F5840008F101084FEA59090437A5E6A000002054
:10F5940000ED00E01AF0010F76D023695FFA89FBD1
:10F5A4001969586B04EB8B0220FA0BF892694FEA45
:10F5B400C81892685FFA88F848EA010808EA02085D
:10F5C40018F0010F1ED05A6B012101FA09F122EA49
:10F5D40001025A633B684FF00108C3F80880584B96
:10F5E4001B6859465B6820469847E378434509D130
:10F5F400B9F1000F06D194F81131042B02D1204641
:10F60400FFF72EFC18F0080F1EBF3B684FF00808E8
:10F61400C3F8088018F0100F1EBF3B684FF01008A5
:10F62400C3F8088018F0400F1EBF3B684FF0400835
:10F63400C3F8088018F0020F1EBF3B684FF00208A1
:10F64400C3F8088018F0800F1ED0D6F83421D6F8FD
:10F6540030319B1AD6F82421934228BF1346033332
:10F664009B0801933B68019A9B699BB2934206D91C
:10F67400D6F83421D6F83031934200D95BB93B68CF
:10F684004FF08008C3F8088009F101094FEA5A0ACB
:10F694000437283631E6A3EB0208D6F82431D6F82D
:10F6A4002811984528BF984608F103039B08019345
:10F6B4005A461FFA88F32046FFF75EF8D6F8283139
:10F6C4004344C6F82831D6F834314344C6F83431BB
:10F6D400C8E747F6F07333423FF485AE4FF028088D
:10F6E40008FB0948C6F30A163246D8F880132046A8
:10F6F400FFF755F8D8F880333344C8F88033D8F886
:10F704008C331E44C8F88C636DE6082204F2CC5195
:10F7140020464FF02808FFF742F808FB0948C6F3D3
:10F724000A16ECE752F8040B8160906B0133816098
:10F7340071E60123A3704023A3800523A0E600BF44
:10F74400A0000020844641EA000313F003036DD1B6
:10F75400403A41D351F8043B40F8043B51F8043B90
:10F7640040F8043B51F8043B40F8043B51F8043B97
:10F7740040F8043B51F8043B40F8043B51F8043B87
:10F7840040F8043B51F8043B40F8043B51F8043B77
:10F7940040F8043B51F8043B40F8043B51F8043B67
:10F7A40040F8043B51F8043B40F8043B51F8043B57
:10F7B40040F8043B51F8043B40F8043B51F8043B47
:10F7C40040F8043B51F8043B40F8043B51F8043B37
:10F7D40040F8043B403ABDD2303211D351F8043BD7
:10F7E40040F8043B51F8043B40F8043B51F8043B17
:10F7F40040F8043B51F8043B40F8043B103AEDD286
:10F804000C3205D351F8043B40F8043B043AF9D2D6
:10F81400043208D0D2071CBF11F8013B00F8013BA9
:10F8240001D30B8803806046704700BF082A13D3B6
:10F834008B078DD010F003038AD0C3F10403D21ACE
:10F84400DB071CBF11F8013B00F8013B80D331F802
:10F85400023B20F8023B7BE7043AD9D3013A11F882
:10F86400013B00F8013BF9D20B7803704B784370ED
:10F874008B78837060467047002103E00A4B5B5825
:10F884004350043109480A4B42189A42F6D3094AB4
:10F8940002E0002342F8043B074B9A42F9D3F9F7FC
:10F8A40097FE00F00DF8704754FB0008000000209C
:10F8B4007405002074050020841E0020FEE700006B
:10F8C40010B562B6F9F7EEFAF9F778F9F9F71EFD13
:10F8D4000020F9F78DF90020F9F7BEFAF9F7FBFCDF
:10F8E400FBF776FDC4B20CB9FAF700F8F8F77EFC22
:10F8F400F8F7EEFF074B02224CB15A83F8F78CFC61
:10F90400F8F7E7FF002CF9D1FAF710F8F6E71A83B5
:10F91400F4E700BF0010024070B4860746D0541EBE
:10F92400002A41D0CAB2034602E014F1FF343BD3AB
:10F9340003F8012B9D07F8D1032C2ED9CDB245EA4B
:10F9440005250F2C45EA054519D903F11002264671
:10F95400103E0F2E42F8105C42F80C5C42F8085C32
:10F9640042F8045C02F11002F2D8A4F1100222F071
:10F974000F0204F00F041032032C13440DD91E4659
:10F984002246043A032A46F8045BFAD8221F22F0DE
:10F9940003020432134404F003042CB1C9B21C441E
:10F9A40003F8011B9C42FBD170BC7047144603460C
:10F9B400C2E700BF024B13B1024800F005B870471C
:10F9C40000000000D9F90008002301461A46184631
:10F9D40000F01EB838B50A4C0A4D641BA4100AD0B6
:10F9E40004F18043013B05EB8305013C55F80439E0
:10F9F4009847002CF9D1BDE8384000F09DB800BF0D
:10FA040054FB000850FB0008704700BF704700BF5C
:10FA14002DE9F8432C4D0646286898460F46914632
:10FA2400FFF7F2FF294B1C68D4F84831002B3ED075
:10FA34005A681F2A1CDC02F1010E76B103EB820125
:10FA44000124C1F88890D3F8880194402043022E01
:10FA5400C3F88801C1F8088123D00232C3F804E056
:10FA6400286843F82270FFF7D1FF0020BDE8F8832F
:10FA7400174B0BB34FF4C870AFF300800346D8B1F3
:10FA8400D4F848210260002141600A46C4F84801C4
:10FA94004FF0010EC0F88811C0F88C11002EDCD094
:10FAA400CCE7D3F88C110C43C3F88C41D5E704F5AB
:10FAB400A673C4F84831BBE72868FFF7A7FF4FF0E7
:10FAC400FF30BDE8F88300BF700500202CFB000860
:10FAD400000000003030313156313030004576615D
:10FAE4006C756174696F6E20446576696365005452
:10FAF40072696E616D6963204D6F74696F6E204326
:10FB04006F6E74726F6C00544D434556414C0056F1
:10FB1400435020436F6E6669670056435020496E18
:10FB2400746572666163650048010020F8B500BF22
:10FB3400F8BC08BC9E467047F8B500BFF8BC08BCCA
:04FB44009E46704722
:08FB4800B9F90008A9810008C9
:04FB500085810008A3
:10FB5400D8FA000812010002020000403C2A000703
:10FB640000020102030104030904000000C20100B1
:10FB740000000800219000082D90000889900008DA
:10FB84006D900008A5900008C1900008DD90000861
:10FB9400419100081D900008439100084591000818
:10FBA40047910008499100081F9000080A060002C6
:10FBB40000000040010000003D9100083990000859
:10FBC400F99000083D90000841900008000E2707B6
:10FBD40000000000000000000102030406070809F9
:10FBE40000000000010203040102030406070809DF
:10FBF400A400002069DF0008B1DE000867DE000809
:10FC0400D7DD000839DE0008BBDD0008A5DD0008EB
:10FC1400E7DD0008F5DD000803DE000819DE000852
:10FC2400FF00000009024300020100C03209040081
:10FC34000001020201000524001001052401000155
:10FC4400042402020524060001070582030800FFBC
:10FC540009040100020A0000000705010240000037
:10FC6400070581024000000011E20008E9E10008F4
:10FC740029E100080000000045E0000865E20008F2
:10FC8400F9E0000881E00008000000000000000026
:10FC940075E00008000000000000000034040020AB
:10FCA4009C04002004050020000000000000000067
:10FCB4000000000000000000000000000000000040
:10FCC4000000000000000000000000000000000030
:10FCD4000000000000000000000000000000000020
:10FCE4000000000000000000000000000000000010
:10FCF4000000000000000000000000000000000000
:10FD040000000000000000000000000000000000EF
:10FD140000000000000000000000000000000000DF
:10FD240000000000000000000000000000000000CF
:10FD340000000000000000000000000000000000BF
:10FD440001000000000000000E33CDAB34126DE65C
:10FD5400ECDE05000B0000000000000000000000C5
:10FD6400000000000000000000000000000000008F
:10FD7400000000000000000000000000000000007F
:10FD8400000000000000000000000000000000006F
:10FD9400000000000000000000000000000000005F
:020000040801F1
:0800C00000000000601E00209A
:040000050800F87D7A
:00000001FF
